:100000000C941E060C9479280C94A6280C94460691
:100010000C9446060C9446060C9446060C94460630
:100020000C9446060C9446060C941B130C9446063E
:100030000C9446060C9446060C9446060C94460610
:100040000C94D3280C9446060C94C12C0C94042DCB
:100050000C9446060C9446060C9446060C944606F0
:100060000C9446060C944606D718391918191B1912
:100070001E192119241927192A19391933196B1A2C
:100080006D1A6D1A6B1A6D1A6D1A6D1A6D1A6D1A3A
:100090006D1A6D1A6D1A6D1A6D1A6D1A6D1A6D1A28
:1000A000F1196D1A6D1A6D1A6D1A6D1A62196D1AA1
:1000B0006D1A6D1A6D1A6D1A6D1A6D1A6D1A6D1A08
:1000C0006D1A6D1A6D1A6D1A6D1A6D1AFD19FD19DA
:1000D000FD19FD19FD19FD19FD19FD19FD196D1AFF
:1000E0006D1A6D1A6D1A6D1A6D1A6219FC19FC19C8
:1000F000FC19FC196D1A0A1A101A161A1C1A221A5F
:10010000281A2E1A341A3E1A481A521A5C1AA319BF
:1001100065196D1A6D1A6D1A6D1AF1196D1A6D1A2D
:100120006D1A6D1A6D1A6D1A6D1A6D1AFB19FB197D
:10013000FB19FB196D1A0A1A101A161A1C1A221A20
:10014000281A2E1A341A3E1A481A521A5C1AA3197F
:1001500065196D1A6D1A6D1A6D1AF119A01AA01A87
:10016000A01AA01AA01AA01AA01AA01AA01AA01ABF
:10017000A01AA01AA01AB71BB71BB71BB71BB71B37
:10018000B71BE51AEF1AF91A031B611B6B1B7A1BCD
:100190008B1B131D281D341D3D1D4C1D711D7A1D0B
:1001A000C31D8C1DD620DC20E220E920F720192178
:1001B0003721456E746572206D656E752E2E2E008A
:1001C000546F67676C6564206D6963726F50504D42
:1001D00000546F67676C656420696E76657274653C
:1001E000642050504D2100546F67676C6564205443
:1001F00058206D7574696E672100546F67676C6570
:10020000642074656C656D65747279210050726F3D
:10021000746F636F6C206572726F72207769746897
:100220002052580054696D656F7574207768656E4B
:1002300020636F6E6E656374696E6720746F205201
:100240005800507265737320616E79206B65792058
:10025000746F2063616E63656C00436F6E6E6563DF
:1002600074696E6720746F2052582C20706F776508
:100270007220757020746865205258202877697440
:10028000682062696E6420706C7567206966206EF4
:100290006F74207573696E6720616C776179732064
:1002A00062696E642900546F67676C656420276912
:1002B0006D6D656469617465206F75747075742700
:1002C00000546F67676C65642027736C61766520E6
:1002D0006D6F64652700546F67676C6564202761E4
:1002E0006C776179732062696E642700546F676769
:1002F0006C65642050504D206368616E6E656C20A3
:100300006C696D69740053657420525353492069B8
:100310006E6A656374696F6E206368616E6E656C8A
:100320002028303D3D64697361626C652900536526
:10033000742050504D206D696E696D756D20737914
:100340006E630053657420626561636F6E20696E31
:1003500074657276616C0053657420626561636FC9
:100360006E2064656C617900536574206265616319
:100370006F6E206672657175656E637920696E2097
:10038000487A3A20303D64697361626C652C205074
:10039000783D504D52206368616E6E656C20782CFC
:1003A0002046783D465253206368616E6E656C202E
:1003B00078005365742050574D2073746F7020641B
:1003C000656C61792028302064697361626C6564B2
:1003D0002C20312D323535203D3D20302E317320FB
:1003E0002D2035306D696E29005365742050504DB5
:1003F0002073746F702064656C61792028302064EC
:10040000697361626C65642C20312D323535203D75
:100410003D20302E3173202D2035306D696E29003E
:10042000536574206661696C736166652064656CF0
:1004300061792028302064697361626C65642C20C6
:10044000312D323535203D3D20302E3173202D2089
:1004500035306D696E29002A2A2A2A2A2A2A2A2A50
:100460002A2A2A2A2A2A2A2A2A2A2A2A2A2A2A2AEC
:100470002A2A2A2A0052582041636B6564202D20C5
:1004800072657665727420737563636573736675E0
:100490006C21002A2A2A2A2A2A2A2A2A2A2A2A2AAD
:1004A0002A2A2A2A2A2A2A2A2A2A2A2A2A2A2A2AAC
:1004B000002A2A2A2A2A2A2A2A2A2A2A2A2A2A2AC6
:1004C0002A2A2A2A2A2A2A2A2A2A2A2A2A2A00528E
:1004D000582041636B6564202D20757064617465DC
:1004E000207375636365737366756C21002A2A2A0D
:1004F0002A2A2A2A2A2A2A2A2A2A2A2A2A2A2A2A5C
:100500002A2A2A2A2A2A2A2A2A2A0056616C696457
:100510002063686F69636573206172653A205B319F
:100520005D2D5B31365D20286368616E6E656C20E1
:10053000312D31362900536574206F7574707574D0
:1005400020666F7220706F727420005B585D2061AE
:10055000626F7274206368616E67657320616E6498
:10056000206578697420525820636F6E6669670051
:100570005B535D20736176652073657474696E6783
:100580007320746F205258005B525D20726576654F
:1005900072742052582073657474696E6773207486
:1005A0006F2064656661756C747300557365206EA9
:1005B000756D62657273205B312D445D20746F2010
:1005C0006564697420706F727473205B452D515D92
:1005D00020666F722073657474696E677300202DD6
:1005E00020726563656976657220636F6E66696700
:1005F000757261746F722C20727820737720000AF4
:100600000A6F70656E4C52536E67200053657420FC
:1006100073657269616C2062617564726174653AB8
:10062000200056616C69642063686F696365733A82
:100630002031202D20342B34202F2032202D203823
:10064000202F2033202D20382B34202F2034202D14
:10065000203132202F2035202D2031322B34202FF5
:100660002036202D20313600536574204368616E9A
:100670006E656C20636F6E6669673A20005365741F
:100680002044617461726174652028302D32293AEA
:10069000200053657420486F70206368616E6E653A
:1006A0006C7320286D61782032342C207365706162
:1006B000726174656420627920636F6D6D61732966
:1006C0002076616C69642076616C75657320312DCC
:1006D0003235353A2000536574206368616E6E656B
:1006E0006C2073706163696E6720287831306B48C5
:1006F0007A293A200053657420524620706F77653E
:10070000722028302D37293A200053657420524634
:10071000206D6167696320286865782920652E67E8
:100720002E20307844454144463030443A2000532E
:1007300065742062617365206672657175656E63AC
:10074000792028696E20487A293A20005B5A5D207A
:10075000656E746572207265636569766572206383
:100760006F6E66696775726174696F6E2075746902
:100770006C79005B465D20646973706C61792061FF
:10078000637475616C206672657175656E63696509
:10079000732075736564005B525D2063616C6375E3
:1007A0006C6174652072616E646F6D206B65792079
:1007B000616E6420686F70206C697374005B495DC2
:1007C000207265696E697469616C697A6520736508
:1007D0007474696E677320746F20736B65746368DB
:1007E0002064656661756C7473005B585D2072658A
:1007F00076657274206368616E67657320616E64EC
:100800002065786974206D656E75005B535D20739B
:100810006176652073657474696E677320746F20E8
:10082000454550524F4D20616E64206578697420B3
:100830006D656E7500557365206E756D62657273BA
:10084000205B302D395D20746F20656469742070E1
:100850006172616D657465727300202D2053797328
:1008600074656D20636F6E66696775726174696F18
:100870006E000A0A6F70656E4C52536E672000510D
:1008800029204F7574707574206265666F726520DB
:100890006C696E6B20283D465329203A2000502970
:1008A00020536C617665206D6F64652028657870D3
:1008B0006572696D656E74616C293A20004F29205C
:1008C00054696D65642042494E44206174207374FC
:1008D000617274757020203A20004E292050504DCE
:1008E000206F7574707574206C696D69746564200F
:1008F000202020203A200044495341424C454400E6
:100900004D292050504D205253534920746F20637D
:1009100068616E6E656C202020203A20004C2920F2
:1009200050504D206D696E696D756D2073796E63E1
:10093000202875732920203A200044495341424C15
:100940004544004B29204661696C736166652062ED
:100950006561636F6E20696E74762E2028312D32AA
:10096000353573293A20004A29204661696C736144
:10097000666520626561636F6E2064656C617920D5
:1009800028302D323535203D3E20313073202D204A
:100990003135306D696E293A200049292046616958
:1009A0006C7361666520626561636F6E206672714B
:1009B0002E203A200048292050574D2073746F7024
:1009C0002064656C6179202020202020203A2000BE
:1009D00047292050504D2073746F702064656C61FE
:1009E00079202020202020203A200046292046611E
:1009F000696C736166652064656C617920202020D4
:100A00002020203A200050574D206368616E6E65AB
:100A10006C200066756E6374696F6E3A2000292041
:100A2000706F72742000506F776572546F776572C3
:100A300000445446205548462033322D62697420C4
:100A400031306368004F70656E4C52536E67525878
:100A5000206D696E6920342F36636800466C7974A6
:100A6000726F6E2F4F72616E6765525820554846FF
:100A70002038636800525820747970653A20004429
:100A8000697361626C656400487A00203D3D200016
:100A900043616C63756C61746564207061636B6540
:100AA0007420696E74657276616C3A200042292068
:100AB0004D6963726F202868616C66292050504D23
:100AC000202020203A00412920496E766572746505
:100AD000642050504D20696E20202020203A0030A4
:100AE00029204D7574652062757A7A657220286DAB
:100AF0006F73746C79293A003929205365726961E2
:100B00006C2062617564726174653A00736D617224
:100B100074506F7274004672536B79005472616E38
:100B200073706172656E740044697361626C6564B0
:100B30000038292054656C656D657472793A2020FF
:100B40002020202020003729204368616E6E656CCC
:100B500020636F6E6669673A202000362920446161
:100B60007461726174652028302D32293A2020206A
:100B700000352920486F70206368616E6E656C7364
:100B80003A2020202020003429204368616E6E65C1
:100B90006C2073706163696E673A202000332920EE
:100BA000524620706F7765722028302D37293A2001
:100BB0002020003229205246206D616769633A2067
:100BC0002020202020202020003129204261736530
:100BD000206672657175656E63793A202020000089
:100BE00000000700020100000304060000000000EE
:100BF00000000001020408102040800102040810D7
:100C00002001020408102004040404040404040263
:100C10000202020202030303030303000000002395
:100C2000002600290000000000250028002B0000FD
:100C3000000000240027002A0000F22D11241FBE0E
:100C4000CFEFD8E0DEBFCDBF13E0A0E0B1E0E2EF30
:100C5000F1E602C005900D92A83CB107D9F716E065
:100C6000A8ECB3E001C01D92AE38B107E1F71CE07B
:100C7000CCE3DCE004C02297FE010E94FB2ECA33C5
:100C8000D107C9F70E942E2E0C94F7300C94000067
:100C900080917305813019F482E08093730580910F
:100CA0007305833019F484E0809373050895A89543
:100CB0000895DC01ED91FC910190F081E02D099502
:100CC00008952091740530917505382748E0C901D1
:100CD000880F991F37FF06C09C0151E2252750E17C
:100CE000352701C09C01415091F730937505209341
:100CF0007405089588E38093760580E092ECA1E086
:100D0000B0E08093770590937805A0937905B09330
:100D10007A0587E08093830580EC9AECA9E8B6E336
:100D200080937B0590937C05A0937D05B0937E0511
:100D300085E0809384058DEE9EEFADEABEED809355
:100D40007F0590938005A0938105B0938205E5E827
:100D5000F5E080E090E0863028F4DC01AE54BC4F32
:100D60002C9101C020E0219301968831910599F7DB
:100D700082E080939D058AE080939E05089580EC33
:100D800097EFAAEBB7E38093BB059093BC05A093C4
:100D9000BD05B093BE0580E090E0A0E0B0E5809393
:100DA000BF059093C005A093C105B093C205E3ECC5
:100DB000F5E080E081938F5F8031E1F70895A0E056
:100DC000B0E0E5EEF6E00C94C42ED82F0E9429295D
:100DD0006115710581059105C9F30E94672F109275
:100DE0007F05109280051092810510928205C4E063
:100DF000812C912C54018A94C0907F05D09080055D
:100E0000E0908105F0908205FE2CED2CDC2CCC24AA
:100E10000E94622FA50194010E94A32E6C0D7D1DDE
:100E20008E1D9F1D60937F057093800580938105C3
:100E300090938205C15001F7DD2309F450C005E805
:100E400015E0E801A12CB12C62E3C62ED12CE12CD7
:100E5000F12C8881882309F442C0B39419F40E94CC
:100E60007A063DC00E94622FA70196010E94A32E20
:100E7000E1E0E60FA5E8B5E08A2F801B8A1520F493
:100E80008D918E13F9CFE9CF2091840530E0A0E158
:100E9000B7E20E943B2E9B01AC01AE2FB0E00E9456
:100EA0004A2E40907B0550907C0560907D057090A7
:100EB0007E05640D751D861D971D4090BB055090E5
:100EC000BC056090BD057090BE05461657066806C5
:100ED000790618F2E993A39488E1A812BACFCDB7A6
:100EE000DEB7E0E10C94E02E8436910520F4BC01DD
:100EF00080E090E017C09C018E3B910528F42A55B4
:100F00003109AAE0B0E00CC0823D910528F4245BD1
:100F10003109A4E6B0E004C02D5C3109A8E5B2E0D7
:100F20000E943B2EA4E6B0E09B01AC010E944A2E39
:100F3000089590E08C599F4F0E947407089582E0B5
:100F40008093B00085E08093B10061E083E00E946F
:100F5000D62960E083E00E940F2A08950097C9F027
:100F60009C0140E050E068E478EE81E090E00E946F
:100F7000A32E2F3F31054105510529F020F02FEF19
:100F800030E040E050E02093B3008091B0008061F9
:100F900003C08091B0008F7E8093B000089560E020
:100FA0008CE00E94D62961E08BE00E94D62961E0A6
:100FB0008DE00E94D62960E082E00E94D62961E09F
:100FC00084E00E94D629089542E050E068E476E08B
:100FD00080E00E9459280895E3E0F0E089E08093E2
:100FE0005700E491E67081E0E63009F080E0089572
:100FF000CF93DF93C82F0E94EC07882381F0DFB7DF
:1010000081E080937205F8940E94570688E18093EE
:101010006000C0936000C1110E945706DFBFDF91DE
:10102000CF9108958F929F92AF92BF92CF92DF920D
:10103000EF92FF92CF93FC01C0A5EC2FE770F0E098
:10104000E658FC4FA081B0E0C7FF03C024E130E0C8
:1010500002C02FE030E0FC0197A183E1989FF001EE
:101060001124E25CFE4F80809180A280B380A20FA9
:10107000B31F20E43FE14DE750E00E94552EA5014B
:1010800094010E94812E8C2F887149F469017A01A4
:10109000E0EDCE0EE7E0DE1EE11CF11C1BC0C7FF39
:1010A00005C060E47AE88CE29EE004C060E07EEE79
:1010B0008AEB9BE069017A01F8EBCF0EFBE0DF1EC3
:1010C000E11CF11CA50194010E94812EC20ED31EC9
:1010D000E41EF51EC701B60169517C4F8F4F9F4F2B
:1010E00028EE33E040E050E00E94812EA8EEB3E00D
:1010F0000E944A2ECF91FF90EF90DF90CF90BF904B
:10110000AF909F908F9008958F3F910551F048F0D8
:10111000811522E0920738F08115934030F482E087
:10112000089580E0089581E0089583E00895A0E0A7
:10113000B0E0EDE9F8E00C94CD2EEB018A01B82F78
:10114000B695A0E028813981F80120832A813B816E
:1011500021832C813D8122832E813F8123836881DD
:1011600079814A815B812C813D81EE81FF819F2FB6
:101170009295990F990F907C272F2370922B252FF2
:101180002370220F220F922B232F23702295207F72
:10119000922BF80194830B5F1F4F2896AF5FBA170D
:1011A00088F680FF24C0888199810E948408D82E07
:1011B0008A819B810E948408E82E8C819D810E94F7
:1011C0008408F82E8E819F810E948408F0E4DF9EBF
:1011D000A001112490E1E99E90011124242B282BD9
:1011E000E4E0FE9EB0011124262BF8012083CDB748
:1011F000DEB7E7E00C94E92E803223E0920708F195
:10120000883E23E0920740F48F519340E4E09695A6
:101210008795EA95E1F70895803D27E0920718F455
:101220008C5D93400895883928E0920768F4885CC3
:10123000974074E0969587957A95E1F78D509C4F8D
:10124000089580E090E008958FEF93E008958C304A
:10125000910540F4A4E0880F991FAA95E1F7885DF5
:101260009C4F0895843F23E0920718F484529C4FCA
:101270000895811524E0920740F48657934FF4E0D7
:10128000880F991FFA95E1F7089580E998E008958D
:101290009C013695279525753575821B930B9C010E
:1012A0002373337396958795969587958373937378
:1012B000820F931F9C0154E0369527955A95E1F7CC
:1012C000280F391F2F703F7041E051E0249FC0016B
:1012D000259F900D349F900D1124892F08952D98EE
:1012E000882319F000002B9A02C000002B98000000
:1012F0002D9A000008952D9A000083B12D980000CA
:10130000829581700895CF93DF93D82F5C9A2D98A2
:101310005C98C8E08D2F80780E946F09DD0FC15066
:10132000C9F72D98DF91CF9108958F770E94830997
:101330000895CF93DF93D82FC8E08D2F80780E9437
:101340006F09DD0FC150C9F72D98DF91CF91089536
:10135000CF93DF932D98C8E080E0D82FDD0F0E9457
:101360007B098D0FC150C9F7DF91CF9108950E947D
:1013700095090E94A8095C9A0895A1E0B0E0E3EC09
:10138000F9E00C94D22E806869830E9483096981F8
:10139000862F0E9499095C9A2196E2E00C94EE2E29
:1013A000CF93C0917F05C827E82FF0E0EA58FA4FA5
:1013B000678589E70E94BD096C2F8DE30E94BD09F6
:1013C0006C2F82E40E94BD09CF91089586E20E94AD
:1013D000B7090895CF93DF93EC016C818CE10E94F3
:1013E000BD096D818DE10E94BD096E818EE10E9473
:1013F000BD096F8180E20E94BD09688581E20E947B
:10140000BD09698582E20E94BD096A8583E20E9466
:10141000BD096B8584E20E94BD096C8585E20E944E
:10142000BD096D858AE20E94BD096E858EE60E9427
:10143000BD096F858FE60E94BD09688980E70E941B
:10144000BD09698981E70E94BD096A8982E70E9416
:10145000BD09DF91CF910895CF92DF92EF92FF9275
:10146000CF93DF936B017C01C11488E3D8068CE92C
:10147000E8068CE1F80628F5C701B60120E836E950
:1014800048E950E00E94812EE901689760E879E61A
:1014900087E69FEF0E945D2E6C0D7D1D8E1D9F1DAA
:1014A000F2E0660F771F881F991FFA95D1F721E7A1
:1014B00032E040E050E00E94812EF22EE32E80E4E4
:1014C00021C0C701B60120E03DE241E351E00E94A6
:1014D000812EE901689760E073ED8EEC9EEF0E942B
:1014E0005D2E6C0D7D1D8E1D9F1D660F771F881F45
:1014F000991F21E732E040E050E00E94812EF22E59
:10150000E32E80E66C2F6F71680F85E70E94BD099E
:101510006E2D86E70E94BD096F2D87E70E94BD09E9
:10152000DF91CF91FF90EF90DF90CF900895682FDB
:101530008DE60E94BD0908958F929F92AF92BF924F
:10154000CF92DF92EF92FF92CF93DF93D82F61E09B
:1015500089E00E940F2A62E370E080E090E00E9440
:101560004C2960E089E00E940F2A62E370E080E08D
:1015700090E00E944C2983E00E94B7098093710596
:1015800084E00E94B7098093700560E086E00E94C5
:10159000BD0961E087E00E94BD096FE789E00E9414
:1015A000BD0965E08AE00E94BD0965E18BE00E940B
:1015B000BD0962E18CE00E94BD096DEF8DE00E94E3
:1015C000BD0960E08EE00E94BD09DD2319F08BE2C9
:1015D00091E008C020919D0533E1239FC0011124B3
:1015E000825C9E4F0E94EA096CE880E30E94BD097C
:1015F0006FE082E30E94BD0962E483E30E94BD09BB
:1016000080919E0587FF02C064E101C06AE084E327
:101610000E94BD096AE285E30E94BD096DE286E38E
:101620000E94BD0964ED87E30E94BD0960E088E384
:101630000E94BD0960E089E30E94BD09D11109C083
:10164000C0907F05D0908005E0908105F0908205E4
:1016500007C0C5E9CC2EC1ECDC2EED2CCEEDFC2E66
:10166000CAE38F2C9924AA24BB24682D8C2F0E94B6
:10167000BD09682D85E08C0F0E94BD09FE2CED2C64
:10168000DC2CCC24CF5FCE3361F76FEF83E40E9474
:10169000BD096FEF84E40E94BD096FEF85E40E94ED
:1016A000BD096FEF86E40E94BD09DD2311F066E0FD
:1016B00002C0609183058DE60E94BD0960E089E764
:1016C0000E94BD09609184058AE70E94BD0960E01F
:1016D00083E70E94BD0960E084E70E94BD09D11143
:1016E00009C060917B0570917C0580917D0590918A
:1016F0007E0504C060EC7AEC89E896E30E942C0A2F
:10170000DF91CF91FF90EF90DF90CF90BF90AF909F
:101710009F908F90089561E087E00E94BD0964E288
:101720008EE70E94BD0963E088E00E94BD0960E089
:1017300088E00E94BD0965E087E00E94BD0962E083
:1017400085E00E94BD0983E00E94B709809371057E
:1017500084E00E94B70980937005089583E00E9499
:10176000B7098093710584E00E94B70980937005E2
:1017700061E087E00E94BD096AE070E080E090E0EF
:101780000E944C290E948B0B00000895CF92DF929B
:10179000FF920F931F93CF93DF931F92CDB7DEB7C6
:1017A000082F162F8EE399830E94BD09F02EC02EBC
:1017B0009981D92E8C2D8F19811738F4F6016191FA
:1017C0006F018FE70E94BD09F5CF64E085E00E94BC
:1017D000BD0983E00E94B7098093710584E00E94EF
:1017E000B709809370050E94292960936C05709356
:1017F0006D0580936E0590936F0569E087E00E9408
:10180000BD0981E0809373050F90DF91CF911F9107
:101810000F91FF90DF90CF9008950F931F930E9438
:10182000C60B80917305813099F40E94292900919B
:101830006C0510916D0520916E0530916F05601B50
:10184000710B820B930B603A76488140910548F307
:1018500080917305813031F46EE971E082EE95E09C
:101860000E94152B1F910F9108950F931F93809144
:101870007305823021F41092730581E020C08091BD
:1018800073058130D9F40E94292900916C051091CB
:101890006D0520916E0530916F05601B710B820BF9
:1018A000930B613A76488140910540F061E087E012
:1018B0000E94BD091092730582E001C080E01F9173
:1018C0000F910895CF93DF93EC014AE050E06D2F24
:1018D00070E082EE95E00E94E32B6EE282EE95E0EE
:1018E0000E94E72ABE0184E0769567958A95E1F724
:1018F0006F7077274AE050E082EE95E00E94E32B7C
:101900006EE282EE95E00E94E72ABE016F707727B3
:101910004AE050E082EE95E00E94E32BDF91CF9108
:101920000895D82FC0E0CD1780F45E9A64E670E089
:1019300080E090E00E944C295E9864E670E080E0D0
:1019400090E00E944C29CF5FEECF6CE271E080E026
:1019500090E00E944C29E6CF0F931F93CF93DF9323
:10196000EC01062F15E0115051F0CE010E94DE303F
:10197000081741F0602FCE010E94E630F4CF82E0DC
:101980000E94910CDF91CF911F910F910895A0E0DB
:10199000B0E0EDECFCE00C94C42E482E562EC0E0D6
:1019A000D0E0612C712CE12CF12C00E010E0411012
:1019B0000CC06090D40586E4689E3001112459E182
:1019C000E52EF12C0AEB15E01EC091E049120FC084
:1019D0006090D405E6E46E9E30011124FBE16F0EA9
:1019E000711C49E2E42EF12C06E715E00CC082E000
:1019F000481209C028E1622E77247394EE24E39400
:101A0000F12C03ED15E043018C0E9D1E109275051F
:101A1000109274053401A62CA818B12CC3010196AC
:101A20006C01AE14BF04A8F4A00EB11E511006C084
:101A3000C3010E94DE30F501808305C0F50160819D
:101A4000C3010E94AC0CF50180810E946106360141
:101A5000E2CFC301511018C0C3010E94DE30B82E7E
:101A6000C6010E94DE302B2D30E0322F2227282B9A
:101A700080917405909175058217930779F4C0E001
:101A8000D0E05524539493CF3601609175050E94A0
:101A9000AC0C60917405C6010E94AC0CC05EDE4FB8
:101AA000C13E92E0D90708F482CF852DCDB7DEB7CD
:101AB000E0E10C94E02E61E082E00E94C70C089502
:101AC00060E082E00E94C70C8091D305853020F051
:101AD0001092D3050E945B0D8091D3058093D405AD
:101AE000089561E080E00E94C70C61E081E00E94FF
:101AF000C70C089560E080E00E94C70C882351F075
:101B000060E081E00E94C70C882321F08091760577
:101B1000883349F00E94BF060E947A0681E00E9445
:101B2000DF060E94710D0895882319F06AEA71E0BA
:101B300002C06EEA71E082EE95E00E94152B0895D6
:101B4000FF920F931F93CF93DF9369EC7BE082EEBC
:101B500095E00E94C12A40917B0550917C056091DF
:101B60007D0570917E052AE030E082EE95E00E94CE
:101B7000EA2B63EB7BE082EE95E00E94C12A409164
:101B80007F0550918005609181057091820520E16B
:101B900030E082EE95E00E94EA2B6DE97BE082EE78
:101BA00095E00E94C12A4AE050E06091830582EEF0
:101BB00095E00E94122C67E87BE082EE95E00E949F
:101BC000C12A4AE050E06091840582EE95E00E94CF
:101BD000122C61E77BE082EE95E00E94C12AC5E805
:101BE000D5E0F12C8E0188818823A9F0FF2031F007
:101BF00061EB71E082EE95E00E94E42A21964AE0D2
:101C000050E0F801608182EE95E00E94DB2BF394B6
:101C1000F8E1FF12E7CF82EE95E00E94EF2A6BE534
:101C20007BE082EE95E00E94C12A4AE050E060919C
:101C30009D0582EE95E00E94122C66E47BE082EE28
:101C400095E00E94C12AE0919E05E770F0E0EE0F5A
:101C5000FF1FEE57FC4F6081718182EE95E00E947C
:101C6000152B61E37BE082EE95E00E94C12A809112
:101C70009E058871883069F028F4811113C068E2EC
:101C80007BE00CC0803141F0883161F46CE07BE096
:101C900005C06CE17BE002C066E17BE082EE95E08E
:101CA0000E94032B68EF7AE082EE95E00E94C12A41
:101CB00040917705509178056091790570917A058A
:101CC0002AE030E082EE95E00E94EA2B6FED7AE0A8
:101CD00082EE95E00E94C12A8091BF0580710E942A
:101CE000940D66EC7AE082EE95E00E94C12A809124
:101CF000BF0580740E94940D6DEA7AE082EE95E053
:101D00000E94C12A8091BF0580720E94940D60E9F3
:101D10007AE082EE95E00E94C12A86E795E00E9473
:101D20001208AB01BC012AE030E082EE95E00E948F
:101D3000CC2B6BE87AE082EE95E00E94C12A86E720
:101D400095E00E9412089B01AC0160E472E48FE010
:101D500090E00E94812EBA01A9012AE030E082EED3
:101D600095E00E94CC2B68E87AE082EE95E00E9434
:101D7000032BCDB7DEB7E5E00C94EB2E8F929F924C
:101D8000AF92BF92CF92DF92EF92FF92811107C084
:101D90006FE77AE082EE95E00E94032B2FC090E07F
:101DA0000E94740724E630E040E050E00E94812E5B
:101DB000CA01B9012AE030E040E050E00E94812EE3
:101DC00049015A016B017C012AE030E0B501A40110
:101DD00082EE95E00E94CC2B6EE282EE95E00E94AE
:101DE000E72A2AE030E0B701A60182EE95E00E94E2
:101DF000CC2B63E782EE95E00E94272BFF90EF90BB
:101E0000DF90CF90BF90AF909F908F9008951F93D9
:101E1000CF93DF9365E77AE082EE95E00E94C12AD6
:101E200080919F05813041F46CE57AE082EE95E087
:101E30000E94032B10E050C0823019F465E47AE070
:101E4000F5CF843019F461E37AE0F0CF853091F773
:101E500066E27AE0EBCFC12FD0E0C930D1050CF4B7
:101E600041C068E3610F82EE95E00E94E72A6EE1CF
:101E70007AE082EE95E00E94C12ABE016F5F7F4F3B
:101E80004AE050E082EE95E00E94AB2B63E17AE0FD
:101E900082EE95E00E94C12AC156DA4FE981E03214
:101EA00018F566E07AE082EE95E00E94C12A898109
:101EB000803130F06DE673E082EE95E00E94E42A16
:101EC00069816F7070E06F5F7F4F4AE050E082EE93
:101ED00095E00E94B42B1F5F80914805181708F405
:101EE000BACF0FC061E3BECFEF70F0E0EE0FFF1F7F
:101EF000EE56FC4F6081718182EE95E00E94152BB9
:101F0000EACF6BEE79E082EE95E00E94C12A8091E3
:101F1000B7050E94BE0E60ED79E082EE95E00E946A
:101F2000C12A8091B8050E94BE0E65EB79E082EE71
:101F300095E00E94C12A8091B9050E94BE0E6AE90F
:101F400079E082EE95E00E94C12A4091AF05509160
:101F5000B0056091B1057091B2054115510561055B
:101F6000710539F12AE030E082EE95E00E94EA2B1B
:101F700067E679E082EE95E00E94C12A8091B30580
:101F80000E949907AB01BC012AE030E082EE95E0A7
:101F90000E94EA2B63E479E082EE95E00E94C12A78
:101FA0004AE050E06091B40582EE95E00E94122C68
:101FB00006C06AE379E082EE95E00E94032B6DE1B2
:101FC00079E082EE95E00E94C12A6091B50570919A
:101FD000B6054AE050E082EE95E00E94FC2B60E0FE
:101FE00079E082EE95E00E94C12A6091AE056034EE
:101FF00050F470E06F5F7F4F4AE050E082EE95E072
:102000000E94B42B06C067EF78E082EE95E00E9454
:10201000032B6AED78E082EE95E00E94C12A809160
:10202000AD0580FF03C063EB71E002C067EB71E0B8
:1020300082EE95E00E94152B6DEB78E082EE95E044
:102040000E94C12A8091AD0582700E94940D6EE9B4
:1020500078E082EE95E00E94C12A8091AD058470FF
:102060000E94940D6FE778E082EE95E00E94C12A0D
:102070008091AD0588700E94940DDF91CF911F91E2
:1020800008950F931F93CF93DF93209145052F3F22
:10209000A9F56FEF75E082EE95E00E94C12A83E812
:1020A00093E00E94620C6EED75E082EE95E00E9476
:1020B000C12A80914605909147050E94620C6BEA07
:1020C00075E082EE95E00E94032B68E875E082EEF1
:1020D00095E00E94032B60E775E082EE95E00E9498
:1020E000032B6BE475E082EE95E00E94032B82EEF9
:1020F00095E00E94EF2A0E94070F68C012160CF0AC
:1021000065C0332727FD30958091480590E0821700
:1021100093070CF45BC066E375E082EE95E00E94E5
:10212000C12A60914505772767FD70954AE050E028
:1021300082EE95E00E94B42B6BE075E082EE95E0B4
:102140000E94C12A10E008E2809149051817D0F5D5
:10215000C12FD0E0CC0FDD1FC65BDA4F288130E005
:1021600080914505992787FD909501972817390794
:1021700039F56BEB71E082EE95E00E94E42A4AE0CB
:1021800050E0602F82EE95E00E94DB2B6FEB71E058
:1021900082EE95E00E94E42AE981EF70F0E0EE0F14
:1021A000FF1FEE56FC4F6081718182EE95E00E9428
:1021B000E42A63EC71E082EE95E00E94E42A0F5F6E
:1021C0001F5FC2CF82EE95E00E94EF2ADF91CF9190
:1021D0001F910F910895FF920F931F93CF93DF9359
:1021E000C5E8D5E0F12C8E0188818823D1F165EC1A
:1021F00071E082EE95E00E94E42A4AE050E06F2D03
:1022000082EE95E00E94DB2B62ED71E082EE95E0BC
:102210000E94E42A2196F801208130E0A0E1B7E293
:102220000E943B2E9B01AC01A0918405B0E00E946E
:102230004A2EAB01BC0180917B0590917C05A09159
:102240007D05B0917E05480F591F6A1F7B1F2AE04C
:1022500030E082EE95E00E94EA2BF394F8E1FF1261
:10226000C2CFCDB7DEB7E5E00C94EB2E1092DF04C1
:1022700085E6E0EEF4E0DF011D928A95E9F7089526
:10228000CF93C82F8F3719F0883009F045C0E091FF
:10229000DF04EE23D9F1E150E093DF04F0E0E052F7
:1022A000FB4F10826DE070E082EE95E00E945906CF
:1022B000C0E08091DF04C81760F4EC2FF0E0E0523A
:1022C000FB4F608170E082EE95E00E945906CF5F7F
:1022D000F0CF60E270E082EE95E00E9459066DE07A
:1022E00070E082EE95E00E945906C0E08091DF0424
:1022F000C81778F5EC2FF0E0E052FB4F608170E0FA
:1023000082EE95E00E945906CF5FF0CF67E082EE43
:1023100095E00E94E72A1DC08B3119F40E94361106
:102320001AC08D30C1F08A30B1F08091DF0484365C
:1023300068F76C2F70E082EE95E00E945906E091FC
:10234000DF0481E08E0F8093DF04F0E0E052FB4F6A
:10235000C08380E001C081E0CF910895CF93C82F62
:102360000E9429296093C8047093C9048093CA0409
:102370009093CB04C093DD04CC2329F040E051EED0
:1023800060E070E004C040E855E260E070E082EE9A
:1023900095E00E94712DCF9108959091CC04492F22
:1023A0004F7050E0BA016F5F7F4F292F30E0E4E0BB
:1023B00035952795EA95E1F76217730759F0FA0109
:1023C000E353FB4F808381E0890F8F70907F892BCF
:1023D0008093CC0408956EE770E082EE95E00E9451
:1023E00059060895A3E1B1E0E8EFF1E10C94C52EA0
:1023F000E5E8F5E0712C8191882321F0739428E1C0
:102400007212F9CF66ED71E082EE95E00E94152B15
:102410004AE050E0672D82EE95E00E94122C80E0A9
:102420000E949C0A0E948B0B8E010E5F1F4FC12CD5
:10243000D12C7601C39466246A945C2C0E941D29D9
:102440004B015C012091840530E0A0E1B7E20E94DD
:102450003B2E9B01AC01C701B6010E945D2E20916D
:102460007B0530917C0540917D0550917E05620F82
:10247000731F841F951F2091BB053091BC054091AF
:10248000BD055091BE05261737074807590718F4B0
:10249000F801608225C08C2D0E94D00961E070E0B7
:1024A00080E090E00E944C29F80110820E941D29D2
:1024B000681979098A099B09643F71408105910572
:1024C00040F40E94E609F8019081981778F780831C
:1024D000EDCF50FE03C05D985E9A02C05D9A5E9893
:1024E0002FEFC21AD20AE20AF20A0F5F1F4F8FEFD4
:1024F000C816D104E104F10409F09FCFCE019395F1
:10250000FC01D82E7FEF68EC2E2F281B271510F02A
:1025100051E056C0DE01129651E02FEF41E03D91AF
:10252000321710F0322F01C0452F5F5F5F3F11F06F
:10253000232FF5CF4193242F30E0A1E0B0E0AC0F82
:10254000BD1FA20FB31F5C93413079F0DE01A20FD3
:10255000B31F5C93423049F0AFEFBFEFAC0FBD1F2C
:10256000A20FB31F6C934E3F78F6A2E0B0E0AC0F21
:10257000BD1FA20FB31F7C934D3F30F6A3E0B0E028
:10258000AC0FBD1FA20FB31F6C93BECF452F242FDE
:1025900030E0FC01E20FF31F6081AFEFB0E0AC0F61
:1025A000BD1FA20FB31F2C91621748F44150DC01EC
:1025B000A40FB11D2C9120836C934111E8CF5F5F74
:1025C000571520F3372D369520E0231770F4DC01E2
:1025D000A20FB11D4C91522F530FFC01E50FF11DBD
:1025E00050815C9340832E5FF0CFF5E8EF2EF5E04D
:1025F000FF2E8C01802F8D19871598F4F801C1905A
:102600008F014AE050E06C2D82EE95E00E94DB2BBA
:102610006CE282EE95E00E94E72AF701C1927F0109
:10262000E9CF82EE95E00E94EF2A81E0CD5EDE4F99
:10263000EFE00C94E12E1F920F920FB60F9211242F
:102640001F932F933F934F935F936F937F938F933A
:102650009F93AF93BF93CF93DF93EF93FF93C0917B
:102660008600D09187008091870490918804209102
:10267000A904211155C09E01281B390B8091BF056B
:102680009091C005A091C105B091C20585FD02C021
:1026900036952795253C49E03407B8F140910A0169
:1026A00050E060E070E02CE1B695A795979587958E
:1026B0002A95D1F70097A105B10521F481E090E0BA
:1026C000A0E0B0E084179507A607B707D8F480917B
:1026D0000A018F3FB9F040E080910A01481780F469
:1026E000842F90E0880F991FFC01E757FB4F208152
:1026F0003181FC01E55FFE4F318320834F5FECCFDA
:102700001092AA0410920A010BC02D3B82E03807F8
:1027100020F080910A018031D8F08FEF80930A0178
:10272000D0938804C0938704FF91EF91DF91CF91FC
:10273000BF91AF919F918F917F916F915F914F91D9
:102740003F912F911F910F900FBE0F901F901895E2
:1027500010910A0181E0810F80930A01C9010E9452
:10276000FC08E12FF0E0EE0FFF1FE757FB4F9183CE
:102770008083D6CF83E0809380008AE980938100B4
:102780008091BF0586FD05C08091810080648093A3
:1027900081008FEF9FEF9093890080938800809154
:1027A0006F00806280936F000895CF93DF930E9443
:1027B000600D8091D405843039F58FE00E94422A63
:1027C000C1E0D0E0892B11F4C0E0D0E080E10E94AC
:1027D000422A892B19F082E090E002C080E090E06C
:1027E0008C2B9D2B8230910539F08330910539F087
:1027F000019739F481E006C01092D40505C082E04B
:1028000001C083E08093D405DF91CF9108956F30AC
:1028100018F086958058089589E0689F802D1124CE
:102820000895A0E0B0E0E7E1F4E10C94CC2EC82FCD
:102830000E942929009138041091390420913A040A
:1028400030913B046B017C01C01AD10AE20AF30A01
:102850009701860149E8C41643E1D406E104F10476
:1028600010F010923C046093380470933904809304
:102870003A0490933B042091A9048FEF820F823099
:10288000D8F5E0913C04EE2309F44EC1E13011F497
:1028900082E0B8C1E03108F034C181E08E0F80934E
:1028A0003C04F0E0E757FB4FC083803109F0ACC136
:1028B000EBE8F4E0213029F4A181A695A69580816A
:1028C00008C080819181A92FA695A695A695969579
:1028D0008795A03148F4B0E090E0AA0FBB1FA55F38
:1028E000BE4F11969C938E931092AA04329684E068
:1028F000E939F807F9F688C1233009F005C1E091FC
:102900003C04E11104C0CF3009F07EC10DC1E831B3
:1029100048F481E08E0F80933C04F0E0E857FB4FD1
:10292000C08372C1E83109F0ECC0C111EAC040E0D7
:1029300050E0ABE0CA01B3E0880F991FBA95E1F708
:10294000A49F9001A59F300D1124F901E757FB4F7B
:102950006081E1817E2F777075956795FC01EE0FA0
:10296000FF1FE55FFE4F71836083F901E657FB4F60
:10297000B081B695B695B695E181FE2FF295FF0F21
:10298000F07E6F2F6B2BE695E695E6957E2F7770A0
:1029900075956795FC01EE0FFF1FE35FFE4F718396
:1029A0006083F901E557FB4FB081B295B695B695B6
:1029B000B370C181DC2FDD0FDD0F6D2F6B2BC29546
:1029C000C695C695C370E281E170EE0FEE0F7E2FC3
:1029D0007C2B75956795FC01EE0FFF1FE15FFE4FA5
:1029E00071836083F901E357FB4FB081B695E181B4
:1029F000FE2FF795FF27F7956F2F6B2BE6957E2F10
:102A0000777075956795FC01EE0FFF1FEF5EFE4F27
:102A100071836083F901E257FB4FB081B295BF70BB
:102A2000E181FE2FF295F07F6F2F6B2BE295EF7017
:102A30007E2F777075956795FC01EE0FFF1FED5E99
:102A4000FE4F71836083F901E157FB4FB081BB1FDB
:102A5000BB27BB1FC181DC2FDD0F6D2F6B2BCC1F64
:102A6000CC27CC1FE281E370EE0F7E2F7C2B759577
:102A70006795FC01EE0FFF1FEB5EFE4F71836083D5
:102A8000F901EF56FB4FB081B695B695E181FE2F67
:102A9000F295FF0FFF0FF07C6F2F6B2BE695E695FD
:102AA0007E2F777075956795FC01EE0FFF1FE95E2D
:102AB000FE4F71836083F901EE56FB4F2081229512
:102AC000269527703181E32FEE0FEE0FEE0F6E2F5C
:102AD000622B732F72957695777075956795FC01CB
:102AE000EE0FFF1FE75EFE4F718360834F5F5F4F06
:102AF0004230510509F01ECF80919F0483FF109250
:102B0000AA0410923C0480C0243009F07DC060917A
:102B10003C0461110BC0C83AB1F4109275051092D3
:102B2000740588EA0E94610681E06CC0613019F486
:102B3000C093370404C0623031F4C09336048C2F44
:102B40000E9461065AC0E09136042E2F30E0220F19
:102B5000331F462F50E0C9010296841795073CF0B9
:102B6000633268F7FA01EA57FB4FC083E8CF2D5F65
:102B70003F4F8C2F90E0609174057091750542175E
:102B8000530749F4982F8827862797279093750530
:102B90008093740532C06817790769F5809137040E
:102BA000813049F5E13118F080E180933604F090EE
:102BB0003604CAE8D4E000E010E00F15D0F4FE01BE
:102BC0003197808190E0982F88272881822B63E0BD
:102BD000969587956A95E1F70E94FC08F801EE0F3B
:102BE000FF1FE55FFE4F918380830F5F1F4F22968B
:102BF000E4CF1092AA0410923C0480913C048823F4
:102C000019F08F5F80933C04CDB7DEB7E8E00C94F9
:102C1000E82ECF93DF93E82FF0E0E654FA4FE185FA
:102C2000E03150F4F894F0E0EE0FFF1FE55FFE4F47
:102C300080819181789437C0E13131F0E23141F007
:102C4000E03161F582E101C083E10E946B2A2BC073
:102C50008FE00E94422AC1E0D0E0892B11F4C0E04D
:102C6000D0E080E10E94422A892B19F082E090E0B6
:102C700002C080E090E08C2B9D2B8230910541F0CA
:102C80008330910541F0019761F086EA92E00BC034
:102C90008CE090E008C089E591E005C080E092E01A
:102CA00002C084EF93E0DF91CF910895A2E2B0E0FB
:102CB000ECE5F6E10C94C22E9E012F5F3F4F80E1C0
:102CC000D9011D928A95E9F764E072E082EE95E001
:102CD00029A33AA30E94152B0E94AE0B1D8A1E8ABF
:102CE0001F8A188E312C212C00E0812C912C54014C
:102CF00070EC472E7DE9572E78E5672E75E3772E29
:102D0000E0E5CE2EE3ECDE2EE12CF12C84EF91E019
:102D1000A0E0B0E08D8F9E8FAF8FB8A380EC97EFCF
:102D2000AAEBB7E3898F9A8FAB8FBC8F80EC9DE9BC
:102D3000A8E5B5E3898B9A8BAB8BBC8B82EE95E0D3
:102D40000E94292C892B09F4E1C082EE95E00E94B3
:102D5000562C9C0133272C32310509F442C0ACF4C7
:102D60002332310509F0ABC019821A821B821C8202
:102D70001D821E821F82188619861A861B861C8653
:102D80001D861E861F86188A60C02434310529F0EE
:102D90002335310509F4B2C092C064E482EE95E0B7
:102DA0000E94E72A2AE030E040EC5DE968E575E33F
:102DB00082EE95E00E94752B6CE282EE95E00E9417
:102DC000E72A2AE030E040EC57EF6AEB77E382EE47
:102DD00095E00E94752B6CE282EE95E00E94272B15
:102DE000ADCF0F5F043009F0A9CF29813A814B8123
:102DF0005C81A8EEB3E00E944A2E698B7A8B8B8BA4
:102E00009C8B2D813E814F8158850E944A2E698F6F
:102E10007A8F8B8F9C8F29853A854B855C852D8F8A
:102E20003E8F4F8F58A32D853E854F8558890E9430
:102E30004A2E6B017C0160323EE4730781059105E7
:102E400030F462E38CE10E94BD0900E077CF60338B
:102E500045E774078105910510F462E2F3CF603411
:102E60005CE975078105910510F466E2EBCF80E51A
:102E7000C81683ECD806E104F10410F462E1E2CF55
:102E800090E6C9169AEED906E104F10410F465E162
:102E9000D9CFA0E7CA16A1E1DA06A1E0EA06F1045B
:102EA00010F461E0CFCFB0EACB16B6E8DB06B1E0B4
:102EB000EB06F10410F463E0C5CF65E0C3CF10ED7D
:102EC000180F1A3008F03ACFE1E0F0E0EC0FFD1FE8
:102ED00024E0029FE00DF11D112420813181428107
:102EE0005381AAE0B0E00E944A2E610F711D811D3E
:102EF000911D608371838283938320CF49885A8890
:102F00006B887C88812C912C540118CF81149104FA
:102F1000A104B10489F4C301B2010E942C0A61E04A
:102F200070E080E090E00E944C291D8A1E8A1F8A72
:102F3000188E312C22242A948D8D9E8DAF8DB8A1B0
:102F400088169906AA06BB06D0F40E94E6092D89C8
:102F50003E894F89588D280F311D411D511D2D8BE4
:102F60003E8B4F8B588F381608F4382E821508F494
:102F7000282E3FEF831A930AA30AB30A56C0C3014F
:102F8000B20128EE33E040E050E00E94812EBA0109
:102F9000A9012AE030E082EE95E00E94CC2B6CE2A1
:102FA00082EE95E00E94E72A4AE050E0632D82EE2F
:102FB00095E00E94DB2B6CE282EE95E00E94E72A0E
:102FC0006D897E898F89988DA50194010E94812E3B
:102FD000BA01A9012AE030E082EE95E00E94CC2BF4
:102FE0006CE282EE95E00E94E72A4AE050E0622D12
:102FF00082EE95E00E94DB2B6CE282EE95E00E946F
:10300000272B4C0C5D1C6E1C7F1C898D9A8DAB8D03
:10301000BC8D84159505A605B70520F449885A8806
:103020006B887C88812C912C540129893A894B89A1
:103030005C89283E33404105510509F07FCEA296B8
:10304000E2E10C94DE2EACE1B0E0E9E2F8E10C94B0
:10305000CC2E0E9429296B017C0181E00E949C0AF0
:1030600014E703E0198361E0CE0101960E940D0C84
:10307000009373050E948B0B6AEF70E080E090E094
:103080000E944C2980917305833089F482EE95E08B
:103090000E94292C892B59F40E9429296C197D0939
:1030A0008E099F096038734C894C9140D8F2809109
:1030B0007305833009F44FC08FE70E9495090E9481
:1030C000A8098983843511F083E05CC00E94A809B7
:1030D00010924605809347050E94A8092091460555
:1030E00030914705280F311D309347052093460541
:1030F0000E94A809809348050E94A8098093490569
:10310000813110F7F12C0F2D10E08091490590E0EE
:10311000880F991F0817190740F40E94A809F801A1
:10312000E65BFA4F8083F394EECF80E7898361E01A
:10313000CE0101960E940D0C83E0809373050E94DE
:103140008B0B62E370E080E090E00E944C2980915C
:103150007305833011F482E015C08FE70E94950952
:103160000E94A8098983803509F0AECF0FE915E0E8
:103170000E94A809F80181938F01F5E00A3B1F071F
:10318000B9F781E06C96E8E00C94E82E8091450553
:10319000992787FD9095A92FB92FFC013196EB3027
:1031A000F10508F066C0EC5CFF4F0C94F92E62E765
:1031B00078E082EE95E00E94032B83E893E00E9482
:1031C000620C6AE578E082EE95E00E94032B65E3ED
:1031D00078E082EE95E00E94032B6BE078E082EECF
:1031E00095E00E94032B6AEE77E082EE95E00E9464
:1031F000032B6DEB77E082EE95E00E94032B67E9ED
:1032000077E082EE95E00E94032B63E777E082EEA1
:1032100095E00E94032B6CE477E082EE95E00E943B
:10322000032B82EE95E00E94EF2A0E94A00D21C0A0
:103230006FE277E01AC06AE077E017C065EF76E0EA
:1032400014C066ED76E011C062E976E00EC06DE76D
:1032500076E00BC068E676E082EE95E00E94032BF4
:1032600062E276E002C06CE076E082EE95E00E94D9
:10327000032B6AE070E080E090E00E944C2982EE2F
:1032800095E00E94292C892B29F082EE95E00E947E
:10329000562CF5CF0895ACE1B0E0E1E5F9E10C94EE
:1032A000CC2E909145059F3F09F023C1482F50E057
:1032B000FA013A97EF36F10508F00FC1E15CFF4FD4
:1032C0000C94F92E61E172E0A0C06DE172E082EE33
:1032D00095E00E94152B85E789838BE1EFE9F5E006
:1032E000DE01129601900D928A95E1F76CE1CE0114
:1032F00001960E940D0C0E948B0B83E08093730556
:1033000068EC70E080E090E00E944C2980917305A9
:10331000843009F0E2C08FE70E9495090E94A80955
:103320008983853509F0D9C06DEE74E082EE95E0B1
:103330000E94032B6FEC74E082EE95E00E94032B59
:1033400061EB74E096C065E372E082EE95E00E9466
:10335000152B89E6898361E0CE0101960E940D0C50
:103360000E948B0B83E08093730568EC70E080E033
:1033700090E00E944C2980917305843009F0ADC023
:103380008FE70E9495090E94A80989838E010E5F2C
:103390001F4F7E014DE1E40EF11C0E94A809F801C7
:1033A00081938F01EE15FF05C1F78BE1FE01329687
:1033B000AFE9B5E001900D928A95E1F789818934F2
:1033C00009F08BC063E974E082EE95E00E94032B64
:1033D00065E774E082EE95E00E94032B67E574E0F8
:1033E00048C06FE472E082EE95E00E94152B8EEFEC
:1033F0008093450572C08052875080539091480554
:10340000981708F066C06EE572E082EE95E00E94C3
:10341000152B63C084E18093450560E274E029C008
:1034200085E18093450569EE73E023C086E18093D2
:10343000450562EB73E01DC087E18093450568E6B2
:1034400073E017C088E18093450567E573E011C01C
:1034500089E18093450563E473E00BC08AE18093C2
:1034600045056EE273E005C08BE18093450566E09B
:1034700073E082EE95E00E94032B2FC06CEE72E0A9
:1034800082EE95E00E94032B8091AD0591E01DC076
:1034900066ED72E082EE95E00E94032B8091AD050F
:1034A00092E013C061EC72E082EE95E00E94032B83
:1034B0008091AD0594E009C066EA72E082EE95E085
:1034C0000E94032B8091AD0598E089278093AD057C
:1034D0008FEF809345050E94411082EE95E00E9497
:1034E000292C892B09F45BC182EE95E00E94562CB1
:1034F000F4CF0E944011882309F451C18091DF0468
:10350000811104C08FEF8093450541C140E050E038
:1035100060E070E080EE94E00E94702F40914505DD
:10352000042F112707FD1095212F312FF801319716
:10353000EB31F10508F01BC1E255FF4F0C94F92E59
:10354000552747FD50952091480530E02417350751
:103550000CF40DC18B019C010150110921093109A5
:10356000003211052105310558F0C0904905EBE402
:10357000F5E0F12CD12CA8E2EA2E415051090FC000
:10358000FA01E156FA4F61506083D9C0DF0111970B
:103590002C9130E02417350729F0F3943296FC1073
:1035A000F5CFCBC00E2D10E020E030E00617170756
:1035B0002807390741F42081DA01A156BA4F119644
:1035C0002C93DD24D394E394E8CF6F3F71058105FC
:1035D000910511F008F0CBC06093B705B0C06F3F04
:1035E00071058105910511F008F0C1C06093B8051F
:1035F000A6C06F3F71058105910511F008F0B7C0B5
:103600006093B9059CC02091E00420622037E9F462
:1036100040E050E060E070E081EE94E00E94702FA6
:103620009B01AC01DC01CB010197A109B10908970D
:10363000A105B10508F0AEC0A4EDB0E30E944A2E8A
:103640006A5E7C4A8A46954E24C02636E9F440E0FC
:1036500050E060E070E081EE94E00E94702F9B01EA
:10366000AC01DC01CB010197A109B1090797A105C4
:10367000B10508F08FC0A8EAB1E60E944A2E645E48
:103680007C438E46944E05C06115710581059105F8
:1036900079F08B019C01005C1D49284535430130C0
:1036A000FAE51F07F2E62F07F2E03F0708F05FC0D8
:1036B0006093AF057093B0058093B1059093B20508
:1036C0003EC06F3F71058105910511F008F04FC0B4
:1036D0006093B30534C08B019C010150110921098D
:1036E00031090F3F11052105310508F040C06093F5
:1036F000B40525C08B019C01045C194021093109E6
:103700000D344DE114072105310528F47093B605F9
:103710006093B50514C0611571058105910521F40B
:103720008FEF8093AE050BC0613471058105910563
:10373000F0F461506093AE0502C0DD20C1F08091CD
:10374000DE0481111AC080917F0590918005A091BF
:103750008105B09182050196A11DB11D80937F0561
:1037600090938005A0938105B093820506C060E721
:1037700072E082EE95E00E94152B0E9436118FEFC9
:10378000809345056AE082EE95E00E94272B0E9417
:10379000411005C061E070E080E090E07ACF6C9667
:1037A000E8E00C94E82E6AE572E082EE95E00E9473
:1037B000032B62E472E082EE95E00E94032B82EE1E
:1037C00095E00E94292C892B31F082EE95E00E9431
:1037D000562C0E944B190E942318823029F0833006
:1037E00051F46DE072E002C064E272E082EE95E0B6
:1037F0000E94032B08958FEF809345051092DE04FD
:103800000E944110809145058E3F69F082EE95E05F
:103810000E94292C892BB1F382EE95E00E94562C50
:103820000E944B19EFCF08950F931F9310914505F8
:103830001F3F09F0D2C0893409F457C000F588331E
:1038400009F469C058F4803309F477C008F061C006
:103850008B3109F440C08132B1F1B9C0813409F42F
:1038600087C030F4893309F466C0803461F1AFC099
:10387000823409F48EC0863409F448C0A8C0823668
:1038800009F487C078F4883531F128F48235C1F124
:103890008335E1F09CC08A3509F494C0813609F47F
:1038A00067C095C0823761F128F4863679F1893690
:1038B000E1F08DC0883779F08A3709F483C0833707
:1038C00009F085C003C061E172E015C00E94710D6E
:1038D0006EE872E004C00E947A0D68EA72E082EE3F
:1038E00095E00E94152B8EEF70C00E947A060E9410
:1038F000BF0667EC72E082EE95E00E94152B67C070
:1039000081E00E94DF0660EE72E0F5CF0E94EB10CE
:103910005EC080535AC06AEF71E082EE95E00E946B
:10392000032B90919E0588E0890F8871977E892BE3
:1039300080939E051AC089E048C067EE71E082EE70
:1039400095E00E94032B8091BF059091C005A09146
:10395000C105B091C20520E182278093BF059093F5
:10396000C005A093C105B093C205109345052FC0B3
:1039700061ED71E082EE95E00E94032B8091BF051E
:103980009091C005A091C105B091C20540E4842783
:1039900010C060EC71E082EE95E00E94032B8091F4
:1039A000BF059091C005A091C105B091C20520E26C
:1039B00082278093BF059093C005A093C105B09363
:1039C000C20502C00E94D31B8FEF809345058091F2
:1039D00045058E3F09F0D4C0DDC00E944011882308
:1039E00009F4D8C08091DF04811104C08FEF809367
:1039F0004505C6C040E050E060E070E080EE94E035
:103A00000E94702F00914505112707FD1095212F69
:103A1000312FF8013197E930F10508F0B4C0E753D0
:103A2000FF4F0C94F92E8B019C01015C1D49284528
:103A300035430F3F19452246324008F0A4C0609339
:103A40007B0570937C0580937D0590937E0577C000
:103A500060937F0570938005809381059093820524
:103A600081E08093DE046BC06830710581059105AB
:103A700008F089C06093830562C08B019C010150EE
:103A80001109210931090A3011052105310508F014
:103A90007AC06093840553C061EB71E080EE94E0DE
:103AA0000E94AA3010E0009799F00E94843000979D
:103AB00079F0183130F4E12FF0E0EA58FA4F8787B7
:103AC0001F5F61EB71E080E090E00E94AA30EBCFD5
:103AD0001831A8F5E12FF0E0EA58FA4F17861F5F7A
:103AE000F7CF653071058105910508F04CC06093F2
:103AF0009D0525C08B019C01015011092109310947
:103B00000630110521053105F0F520919E05287F2D
:103B1000262B20939E0513C08B019C010150110997
:103B2000210931090115124C2140310560F56093DE
:103B30007705709378058093790590937A05809145
:103B4000DE04811113C080917F0590918005A091C2
:103B50008105B09182050196A11DB11D80937F055D
:103B600090938005A0938105B09382050E94361141
:103B70008FEF809345056AE082EE95E00E94272B47
:103B80000E94C61807C060E772E082EE95E00E94CE
:103B9000152BECCF1F910F9108958FEF8093450562
:103BA0001092DE040E94C618809145058E3F69F090
:103BB00082EE95E00E94292C892BB1F382EE95E0EC
:103BC0000E94562C0E94141CEFCF6AE070E080E047
:103BD00090E00E944C2982EE95E00E94292C892BCE
:103BE00029F082EE95E00E94562CF5CF0895CF93F0
:103BF000C82F682F82EE95E00E94832C90916A0571
:103C00009C2790936A05CF910895A1E0B0E0EBE086
:103C1000FEE10C94D22E99830E94F71D9981892F81
:103C20000E94F71D2196E2E00C94EE2E1F93CF9395
:103C3000DF93182FEB0110926A0565EB70E082EEBE
:103C400095E00E94590662E670E082EE95E00E94DF
:103C50005906812F0E94F71DCE010E94051EDF919B
:103C6000CF911F91089560916A0582EE95E00E94C0
:103C7000832C0895A1E2B0E0E0E4FEE10C94CE2EA6
:103C80007B018A018C3009F453C108F040C08630B2
:103C900009F4BCC018F5833009F491C070F4813088
:103CA00009F472C0823009F048C26BE170E082E032
:103CB0000E94161E0FE915E078C0843009F487C011
:103CC000853009F03AC26091490570E0660F771FB0
:103CD00085E00E94161E0AE415E086C0893009F4CA
:103CE000A7C070F4873009F49BC0883009F025C262
:103CF00061E070E088E00E94161E8091D40523C226
:103D00008A3009F4CAC08B3009F4F2C016C28A3670
:103D100009F475C1D8F4873609F43AC138F4853608
:103D200009F40EC1863609F41FC107C2883609F4AA
:103D300037C1893609F001C261E070E089E60E946E
:103D4000161E0E947A060E94BF06F5C18D3609F440
:103D5000D4C138F48B3609F491C18C3609F49AC178
:103D6000ECC18E3609F4DCC1873C09F0E6C161E0A4
:103D700070E087EC0E94161E81E00E94F71D0E94F1
:103D8000331E10926B05E3C169E270E081E00E948E
:103D9000161E06E715E0F80181918F010E94F71DBC
:103DA000F5E00F391F07B9F7D0C1F80181918F01F4
:103DB0000E94F71DF5E00A3B1F07B9F7C6C161E095
:103DC00070E083E00E94161E0E942318BCC161E0CF
:103DD00070E084E00E94161E81E00E94F71D0E94A0
:103DE000331E0E945616B3C18091490590E0880F9A
:103DF000991F98012A5435402817390708F0A5C1A2
:103E0000F80181918F010E94F71DEECF62E070E012
:103E100086E00E94161E83E893E00E94051E95C16D
:103E200061E070E087E00E94161E809148058BC11A
:103E300086E6898361E0CE0101960E940D0C0E9406
:103E40008B0B83E08093730568EC70E080E090E07A
:103E50000E944C29809173058430D9F48FE70E9429
:103E600095090E94A8098983863469F460E270E0AC
:103E700089E00E94161E10E20E94A8090E94F71D08
:103E80001150D1F762C161E070E089E00E94161E16
:103E900052C161E070E089E053C169E170E08AE0FD
:103EA0000E94161E82E08093BA05209172058091CF
:103EB000BF059091C005A091C105B091C205222314
:103EC00011F0806801C08F778093BF059093C00583
:103ED000A093C105B093C2050AEB15E0F8018191EA
:103EE0008F010E94F71DF5E0033D1F07B9F72DC1B3
:103EF00061E270E08BE00E94161E8091AA048F3F61
:103F000039F08091AA0491E0980F9093AA0402C01E
:103F10008091AA040E94F71D10E0812F0E940916CB
:103F20000E9427090E94051E1F5F1031B1F70DC1C5
:103F300061E070E08CE00E94161E8091D30503C101
:103F400061E070E085E60E94161E89E2E816F10441
:103F500009F0F8C0D801E6E7F5E08D91819385E09E
:103F6000EF39F807D1F7E7C061E070E086E60E941C
:103F7000161EEBE1EE16F10409F0E4C0D801EFE9FA
:103F8000F5E08D91819385E0EA3BF807D1F7D3C046
:103F900061E070E087E60E94161E0E94710DCBC0A2
:103FA00061E070E088E60E94161E85E789838BE158
:103FB000EFE9F5E0DE01129601900D928A95E1F7A6
:103FC0006CE1CE0101960E940D0C0E948B0B83E0E8
:103FD0008093730560E273E080E090E00E944C29DA
:103FE00080917305843009F0ADC08FE70E94950978
:103FF0000E94A8098983853509F0A4C09CC061E0AE
:1040000070E08AE60E94161E89E6898361E0CE018F
:1040100001960E940D0C0E948B0B83E08093730528
:1040200060E273E080E090E00E944C29809173058B
:10403000843009F087C08FE70E9495090E94A80983
:1040400089838E010E5F1F4F7E01EDE1EE0EF11CA4
:104050000E94A809F80181938F01EE15FF05C1F7B1
:104060008BE1FE013296AFE9B5E001900D928A95A1
:10407000E1F78981893409F065C05DC061E070E0D5
:104080008BE60E94161EF80180818093D4050E9461
:104090007A0D51C061E070E08CE60E94161EF0E2DD
:1040A000EF16F10461F487E6898380E2F801DE010E
:1040B000129601900D928A95E1F761E203C087E4C0
:1040C000898361E0CE0101960E940D0C0E948B0B4A
:1040D00083E0809373056CE474E080E090E00E94DC
:1040E0004C2980917305843069F58FE70E9495090A
:1040F0000E94A809873431F51EC061E070E08DE6AA
:104100000E94161E89E1E816F104E1F4D801EAEBF9
:10411000F5E08D91819385E0E33DF807D1F70BC081
:1041200061E070E08EE60E94161EF80180818093A7
:10413000D3050E945B0D81E006C061E070E08AEC6F
:104140000E94161E80E00E94F71D0E94331EA19659
:10415000E6E00C94EA2EA0E0B0E0E1EBF0E20C9493
:10416000CC2ECAECD3E014E606E035E0F32E44E0B2
:10417000E42E53E0D52E62E0C62E82EE95E00E943A
:10418000292C892B09F49BC082EE95E00E94562CC5
:10419000282F809335044091340450E04730510576
:1041A00060F7FA01EE52FF4F0C94F92E853B29F788
:1041B00081E080933404E1CF823609F07DC0C09263
:1041C0003404DBCF8093330480933204D0923404E0
:1041D000D4CF9C0133273093310420933004909145
:1041E0003204982790933204E0923404C6CF382FDB
:1041F00022274091300450913104242B352B3093E9
:104200003104209330049091320498279093320423
:10421000F09234042536310508F4AFCF61E070E048
:104220008CEC0E94161E81E00E94F71D0E94331E36
:1042300043C020912E0430912F04F901E653FC4F26
:10424000808390913204982790933204C90101969B
:1042500090932F0480932E042091300430913104E8
:104260008217930708F489CF0093340486CF809196
:10427000320482130BC060912E0470912F044AEC1B
:1042800053E0809133040E943A1E0DC062E070E05A
:104290008BEC0E94161E809133040E94F71D8091C2
:1042A0006A050E94F71DFE01812F11928A95E9F798
:1042B00010922F0410922E04109234045ECFCDB7CA
:1042C000DEB7E8E00C94E82E81E080936B058091E6
:1042D0006B05882349F082EE95E00E94292C892BFA
:1042E000B1F30E94AB20F3CF0895AAE2B0E0EBE770
:1042F000F1E20C94CA2E0E941D296B017C0181E021
:104300000E949C0A82EE95E00E94292C892B29F0BC
:1043100082EE95E00E94562CF5CF5E9811E072E691
:10432000B72EE9E2AE2E03E00E941D296C197D092B
:104330008E099F09693C710581059105D0F1112312
:10434000C1F10E941D296B017C015D9A80ED97E00F
:104350000E94AE07B982E6E7F5E0DE0112968A2DEB
:1043600001900D928A95E1F76AE2CE0101960E94D2
:104370000D0C5D9880E090E00E94AE0700937305FD
:104380000E948B0B62E370E080E090E00E944C2979
:1043900080917305843061F4009373058FE70E9468
:1043A00095090E94A80911E0823419F410E001C0B7
:1043B00011E08EE00E94422A892B81F411E00EC0A8
:1043C0005E9A5D9A82EE95E00E94562C8D309105A2
:1043D000A9F05CF40A9791F05E985D9882EE95E002
:1043E0000E94292C892B61F79FCF8332910579F0A8
:1043F0008234910589F70E946421EECF62EB71E06F
:1044000082EE95E00E94032B0E94CD1DE5CF0E9415
:104410005616E2CF8F929F92AF92BF92CF92DF92C9
:10442000EF92FF921F93CF93DF938EE00E94422A78
:10443000892B09F089C068EC70E080E090E00E9470
:104440004C2980E090E00E94AE070E941D294B019C
:104450005C016B017C0180ECC80E82E1D81EE11C7E
:10446000F11C0E941D296C157D058E059F0530F4F9
:104470008EE00E94422A892BA1F364C08EE00E9444
:10448000422A892B09F05EC080ED97E00E94AE07BA
:104490000E941D296B017C01D0E0C1E088E4880EF8
:1044A00086E2981EA11CB11C11E08EE00E94422AF7
:1044B000892B21F58C149D04AE04BF0430F480EDEB
:1044C00097E00E94AE07D1E0F0CF0E941D296C1941
:1044D0007D098E099F09693C71058105910528F3C5
:1044E0000E941D296B017C01C12719F080ED97E026
:1044F00002C080E090E00E94AE07D7CF80E090E05D
:104500000E94AE07DD23B9F08091D30590E00196BB
:1045100065E070E00E946D2E8093D3050E945B0DD4
:104520000E94D5130E947A0D64EF71E080E090E064
:104530000E944C2909C080E00E94DF060E94F2110F
:104540000E94710D0E947521DF91CF911F91FF9004
:10455000EF90DF90CF90BF90AF909F908F90089595
:10456000CF92DF92EF92FF9280E00E94F8070E94C4
:10457000CF0761E089E00E94D62960E089E00E94CF
:104580000F2A61E086E00E94D62961E085E00E9462
:10459000D62960E08EE00E94D62960E08FE00E947C
:1045A000D62961E08FE00E940F2A60E080E10E943E
:1045B000D62961E080E10E940F2A60E088E00E9435
:1045C000D62961E088E00E940F2A61E081E10E9423
:1045D000D62960E081E10E940F2A0E949F0740E0F7
:1045E00052EC61E070E082EE95E00E94712D0E9435
:1045F000D5130E947A0D0E94BA138FEF8093AA04FC
:104600000E94E40778940E941D296B017C0180912F
:10461000AA048F3F59F40E941D296C197D098E0947
:104620009F09603D77408105910588F380ED97E013
:104630000E94AE0761E08EE00E940F2A5E9A82EE31
:1046400095E00E94292C892B29F082EE95E00E94AA
:10465000562CF5CF6DEF72E082EE95E00E94E42AD1
:1046600083E893E00E94620C64E173E082EE95E0DF
:104670000E94E42A4AE050E064E070E082EE95E0B7
:104680000E94B42B62E370E080E090E00E944C292D
:1046900082EE95E00E94292C04970CF182EE95E0C1
:1046A0000E94562C82349105D1F482EE95E00E944E
:1046B000562C8E34910599F482EE95E00E94562C8A
:1046C0008434910561F482EE95E00E94562C819726
:1046D00031F480E090E00E94AE070E947521409185
:1046E0007705509178056091790570917A05DB0125
:1046F000CA010197A109B1090497A105B10568F4A0
:104700004093A904433029F440EA56E861E070E0A0
:1047100004C040E052EC61E070E082EE95E00E945F
:10472000712D0E940A225E9880E090E00E94AE0700
:104730000E94BA131092C5048091BF0583FF11C077
:1047400080918B05882351F080919205882331F068
:1047500080919905882311F087E001C085E080935E
:10476000C50480E00E949C0A8091C6040E94D00982
:104770000E948B0B10923F0410923E0410923D0455
:10478000F12C8091D4058F15B0F062E370E080E0E9
:1047900090E00E944C2980ED97E00E94AE0762E312
:1047A00070E080E090E00E944C2980E090E00E9460
:1047B000AE07F394E6CF80919E0584FF08C0982F42
:1047C000987181E0983109F080E00E94AE118FE08D
:1047D0000E94F807FF90EF90DF90CF900895EF923E
:1047E000FF920F931F93CF93DF938C016EE770E0DE
:1047F00082EE95E00E945906E801F12CF0E2EF2EDE
:104800008E0188818D57823048F46DE770E082EE2A
:1048100095E00E94590688818E2588832196F801AB
:10482000608182EE95E00E94832CF394F9E0FF1200
:10483000E7CF6EE770E082EE95E00E945906CDB7B3
:10484000DEB7E6E00C94EA2EA9E0B0E0EAE2F4E29A
:104850000C94D22E9091C70491110EC09EEF9983B3
:104860008A836B8350E0559547954C832D83198639
:1048700018861F821E822EC04091CC04842F90E0A7
:10488000B4E095958795BA95E1F7242F2F7030E025
:104890008217930719F18DEF89831B82FE013496ED
:1048A00050E0842F90E0A4E095958795AA95E1F7D4
:1048B000242F2F7030E08217930749F0DC01A353B7
:1048C000BB4F8C918193405F5F5F563051F74093AF
:1048D000CC045A83CE0101960E94EF238091C70435
:1048E00090E0019666E070E00E946D2E8093C70410
:1048F0002996E2E00C94EE2EA0E0B0E0E2E8F4E2CB
:104900000C94CB2E6C016EE770E082EE95E00E9475
:1049100059068601E12CF12CC0E0D0E030E2B32E44
:10492000F801608183E8860F823078F46DE770E0EB
:1049300082EE95E00E945906F80160816B2570E0D7
:1049400082EE95E00E94590604C082EE95E00E9436
:10495000832CE114F10459F0F80180819E01280FA5
:10496000311DC901C92FDD27C80FD91FDD273FEF32
:10497000E31AF30A89E0E816F10459F028E0E21698
:10498000F10421F48C2F8095F60180870F5F1F4F73
:10499000C7CFCDB7DEB7E9E00C94E72EA9E0B0E0D1
:1049A000E4EDF4E20C94D22EE82F362F8091C70468
:1049B00090E0019664E270E00E946D2E8093C7043F
:1049C00058E9598350E15A83813089F048F08230A8
:1049D000B9F08330D9F48B8381EF8C833D8319C088
:1049E00085E08B8381EF8C832F5F2D8312C08B83B7
:1049F00081EF8C8384E6489FA00111245D8309C068
:104A000084E08B8381EF8C83ED8303C00E94EB11E4
:104A100004C0CE0101960E947C242996E2E00C9409
:104A2000EE2EA2E0B0E0E7E1F5E20C94C72E182FDD
:104A3000762E2A8349830E9429296B017C0180916B
:104A4000DD048090C8049090C904A090CA04B0907E
:104A5000CB042A8149818823C1F0D701C601881976
:104A60009909AA09BB094C015D0191EE89169EE2E4
:104A70009906A104B10420F1241708F4422F202F35
:104A8000672D812F0E94CE2413C0D701C60188193B
:104A90009909AA09BB094C015D0191E3891695E7C3
:104AA0009906A104B10460F0672D812F0E9424248F
:104AB000C092C804D092C904E092CA04F092CB0418
:104AC0002296EDE00C94E32EA2E2B0E0EAE6F5E2F5
:104AD0000C94C82E8CE00E94B70981110DC06CE1C6
:104AE00073E082EE95E00E94152B5E9A80E00E94B2
:104AF0009C0A0E948B0B5E9882EE95E00E94292C06
:104B0000892B01F182EE95E00E94562C9091A90428
:104B1000992319F00E941114EFCF40913E0450E008
:104B20009A012F5F3F4F2F71332760913F0470E050
:104B30002617370709F3FA01E75BFB4F80832093C1
:104B40003E04DACF80917305843009F086C00E945C
:104B50002929611571058105910549F06093B70414
:104B60007093B8048093B9049093BA040CC081E0A8
:104B700090E0A0E0B0E08093B7049093B804A093D5
:104B8000B904B093BA048091AD049091AE048160F1
:104B90009093AE048093AD0483E0809373058FE718
:104BA0000E94950909E614E00E94A809F801819382
:104BB0008F01F4E002371F07B9F72091720480914A
:104BC0006904982F922796FF3BC090E49227909318
:104BD0007204982F98739833F1F410E0212F30E08D
:104BE00080916904877090E0821793074CF11F5FF2
:104BF00020919E05812F90E0FC01E759FB4F24FF97
:104C000004C080810E94CD11E9CF608182EE95E0E1
:104C10000E94832CE3CF8F7399F480916A04809370
:104C2000B60480916B048093B40480916C048093EB
:104C3000B30480916F0490E09093AC048093AB0434
:104C400080913D04813019F482E080933D0480918D
:104C50003D04833011F410923D040E9429296B0118
:104C60007C018091AF049091B004A091B104B09107
:104C7000B2040097A105B105C9F0A7019601281B50
:104C8000390B4A0B5B0BDA01C901883B9B40A1053C
:104C9000B10560F00E94E6098093B5041092AF045C
:104CA0001092B0041092B1041092B2048091BB042F
:104CB0009091BC04A091BD04B091BE04460157017F
:104CC000881A990AAA0ABB0A86E795E00E94120888
:104CD00086169706A806B90608F4B1C0C092BB04B0
:104CE000D092BC04E092BD04F092BE040E9457062C
:104CF0008091AA048830A0F08091BF059091C005F2
:104D0000A091C105B091C2055CE1B695A7959795B4
:104D100087955A95D1F7892B8A2B8B2B09F0B8C12F
:104D20008091AA048F5F8093AA048091B704909128
:104D3000B804A091B904B091BA040097A105B105D7
:104D4000F1F0C81AD90AEA0AFB0A86E795E00E9440
:104D500012086C157D058E059F0508F00FC1809126
:104D6000BF0584FD04C080ED97E00E94AE0710925D
:104D7000B7041092B8041092B9041092BA0490913A
:104D80007204907C9093720450913E0480913F0491
:104D900020913D04581709F40EC1223009F00BC1CF
:104DA000905890937204E0919E05E770F0E0E65809
:104DB000FC4F6081693008F0E6C0615040E0461366
:104DC000E4C080933F0487E3840F90917204892BA1
:104DD000809372044093400483E080933D045D9A85
:104DE000109183058091C504811132C18091BF0566
:104DF00082FD3AC1812F0E94970A8091C6040E94C9
:104E0000D009E0919E05E770F0E0E658FC4F608124
:104E100082E794E00E94C60B8091BF0582FD2DC100
:104E2000E091C604EF5FE093C604E83109F42DC1B8
:104E3000F0E0EA58FA4F8785882309F426C10E94DA
:104E4000350C813069F580919E05887149F180911A
:104E5000AD049091AE04880F991F9093AE04809397
:104E6000AD0483E0809373050E948B0B0E94292977
:104E70006093AF047093B0048093B1049093B20434
:104E8000672B682B692B61F481E090E0A0E0B0E033
:104E90008093AF049093B004A093B104B093B20494
:104EA00080919E0584FF1FC08091AD049091AE0457
:104EB0008E7F0E944809182F6091AB048091B60440
:104EC0000E940714482F612F8091B50449A30E94C6
:104ED00007140091D405282F49A16091B304809153
:104EE000B4040E9411255D988091C3048130C1F003
:104EF00018F08230B1F1D9C08EE00E94422A892B8D
:104F000009F0D3C081E08093C3040E941D296093FF
:104F1000BF047093C0048093C1049093C204C5C0C1
:104F20008EE00E94422A892B31F50E941D29C090F3
:104F3000BF04D090C004E090C104F090C2046C198A
:104F40007D098E099F09693E73408105910508F42A
:104F5000ACC082E08093C30480ED97E00E94AE076E
:104F6000A4C08EE00E94422A892B09F49EC080E0F2
:104F700090E00E94AE071092C30497C080E090E0DA
:104F80000E94AE07FCCE68E019CF851709F419CF4F
:104F90004F5F242F30E090E0F901EE58FB4FDC0129
:104FA000A75BBB4F7C917083F901E05CFB4F708382
:104FB00001968F7104CF2430B1F42091400481E434
:104FC00094E0A3E7B4E0FC013E2F381B321718F43D
:104FD00031913D93F9CF87E3820F90917204892B31
:104FE00080937204F9CE8091C304823051F49160B1
:104FF000909372045E9A8E010F5F1F4FF12CB801DF
:1050000010C05E9880913D04811103C081E08093BF
:105010003D0480913D04833071F784E080933D042A
:10502000EACF8F2D69A37AA30E940916F801819314
:1050300091938F01F39469A17AA1F0E1FF12F1CF6E
:1050400080919E0543E754E087700E949708C7CE81
:10505000112309F4CBCE9091C40421E0290F2093B1
:10506000C4049813C3CE1DC08FE00E94422A892B2E
:1050700009F0C0CE5E9A17E0BDCE8FE00E94422AB2
:10508000892B09F0CDCE5E98CBCE1092C604D7CE38
:105090008091AA04883009F45E9A89E08093AA047A
:1050A000CECE1092C4041150A1CEA296ECE00C9486
:1050B000E42E8230E8F4E82FF0E0EE0FFF1FEB5211
:1050C000FA4F71836083813041F0809169008C7F59
:1050D000842B80936900E89A089580916900440FB9
:1050E000551F440F551F837F842B80936900E99AD5
:1050F00008951F920F920FB60F9211242F933F9392
:105100004F935F936F937F938F939F93AF93BF93CF
:10511000EF93FF938091D5059091D605892B29F0C7
:10512000E091D505F091D6050995FF91EF91BF91DA
:10513000AF919F918F917F916F915F914F913F912F
:105140002F910F900FBE0F901F9018951F920F92E6
:105150000FB60F9211242F933F934F935F936F934A
:105160007F938F939F93AF93BF93EF93FF93809120
:10517000D7059091D805892B29F0E091D705F091BA
:10518000D8050995FF91EF91BF91AF919F918F91B4
:105190007F916F915F914F913F912F910F900FBE33
:1051A0000F901F9018951F920F920FB60F92112417
:1051B0002F933F938F939F93AF93BF938091DA0583
:1051C0009091DB05A091DC05B091DD053091D9050A
:1051D00023E0230F2D3720F40196A11DB11D05C03A
:1051E00026E8230F0296A11DB11D2093D9058093B7
:1051F000DA059093DB05A093DC05B093DD05809183
:10520000DE059091DF05A091E005B091E1050196E2
:10521000A11DB11D8093DE059093DF05A093E005ED
:10522000B093E105BF91AF919F918F913F912F91E5
:105230000F900FBE0F901F9018952FB7F8946091A4
:10524000DA057091DB058091DC059091DD052FBFBB
:1052500008953FB7F8948091DE059091DF05A09105
:10526000E005B091E10526B5A89B05C02F3F19F0D8
:105270000196A11DB11D3FBF6627782F892F9A2F58
:10528000620F711D811D911D42E0660F771F881FFF
:10529000991F4A95D1F70895CF92DF92EF92FF922E
:1052A000CF93DF936B017C010E942929EB01C1148C
:1052B000D104E104F10479F00E9429296C1B7D0BD3
:1052C000683E7340A0F381E0C81AD108E108F108F4
:1052D000C851DC4FECCFDF91CF91FF90EF90DF9082
:1052E000CF900895789484B5826084BD84B5816040
:1052F00084BD85B5826085BD85B5816085BDEEE6DE
:10530000F0E0808181608083E1E8F0E010828081BC
:1053100082608083808181608083E0E8F0E080812A
:1053200081608083E1EBF0E0808184608083E0EB4A
:10533000F0E0808181608083EAE7F0E08081846032
:10534000808380818260808380818160808380818E
:10535000806880831092C1000895833081F028F422
:10536000813099F08230A1F008958630A9F087301D
:10537000B9F08430D1F4809180008F7D03C080919A
:1053800080008F7780938000089584B58F7702C066
:1053900084B58F7D84BD08958091B0008F7703C060
:1053A0008091B0008F7D8093B0000895CF93DF93FC
:1053B00090E0FC01ED50F44F2491FC01E95FF34FC4
:1053C0008491882349F190E0880F991FFC01E15DE9
:1053D000F34FA591B4918B5D934FFC01C591D4918E
:1053E0009FB7611108C0F8948C91209582238C930B
:1053F000888182230AC0623051F4F8948C91322F54
:10540000309583238C938881822B888304C0F89401
:105410008C91822B8C939FBFDF91CF910895A1E057
:10542000B0E0E5E1FAE20C94D02E282F30E0F9014B
:10543000E152F44F8491F901ED50F44F1491F901C8
:10544000E95FF34F04910023C9F0882321F06983B9
:105450000E94AD296981E02FF0E0EE0FFF1FEB5DA8
:10546000F34FA591B4919FB7F8948C91611103C04B
:105470001095812301C0812B8C939FBF2196E4E07E
:105480000C94EC2ECF93DF93282F30E0F901E152FA
:10549000F44F8491F901ED50F44FD491F901E95F93
:1054A000F34FC491CC2391F081110E94AD29EC2FD0
:1054B000F0E0EE0FFF1FE55EF34FA591B4912C9144
:1054C0002D2381E090E021F480E002C080E090E0B4
:1054D000DF91CF9108958E3008F08E508770209123
:1054E0009D0190E4299F90011124822B80937C00E0
:1054F00080917A00806480937A0080917A0086FDA2
:10550000FCCF809178002091790090E0922B089553
:10551000A0E0B0E0EEE8FAE20C94CC2E6C017A0147
:10552000EB01E60EF71E00E010E0CE15DF0561F09E
:105530006991D601ED91FC910190F081E02DC601B9
:105540000995080F191FF1CFC801CDB7DEB7E8E004
:105550000C94E82E6115710589F0DB010D90002097
:10556000E9F7AD0141505109461B570BDC01ED91A4
:10557000FC910280F381E02D0995089580E090E090
:105580000895EF92FF920F931F93CF93DF938C01B7
:10559000FB01C0E0D0E064917F018FEFE81AF80AC8
:1055A000662361F0D801ED91FC910190F081E02D2E
:1055B000C8010995C80FD91FF701EDCFCE01CDB7AE
:1055C000DEB7E6E00C94EA2E0E94AA2A0895DC01D8
:1055D000ED91FC910190F081E02D099508950F93D4
:1055E0001F93CF93DF93EC016DE00E94E72A8C01BB
:1055F0006AE0CE010E94E72A800F911FDF91CF91D0
:105600001F910F9108950F931F93CF93DF93EC0198
:105610000E94C12A8C01CE010E94EF2A800F911FA7
:10562000DF91CF911F910F9108950F931F93CF9307
:10563000DF93EC010E94AA2A8C01CE010E94EF2A7E
:10564000800F911FDF91CF911F910F9108950F93BC
:105650001F93CF93DF93EC010E94E72A8C01CE01C8
:105660000E94EF2A800F911FDF91CF911F910F9120
:105670000895A1E2B0E0EFE3FBE20C94C82E7C01B8
:10568000C42EE52FCB01D22E19A221E02D1510F04A
:105690002AE0D22E8E010F5D1F4F8D2C912CA12C54
:1056A000B12C6C2D7E2FA50194010E94812E8C2D92
:1056B000D29E80191124015011098A3010F4805DA6
:1056C00001C0895CF8018083211531054105510530
:1056D00021F0C22EE32FCA01E4CFB801C7010E9416
:1056E000AA2AA196ECE00C94E42EA0E0B0E0EBE74F
:1056F000FBE20C94CC2EEC016A017B0121153105F3
:1057000041F4E881F9810190F081E02D642F099541
:105710001DC02A303105A9F477FF12C06DE20E9446
:10572000E72A8C0144275527BA014C195D096E09F7
:105730007F092AE0CE010E94392B800F911F06C0FD
:105740002AE0B701A601CE010E94392BCDB7DEB702
:10575000E8E00C94E82E9A01AB01662757FD6095AE
:10576000762F0E94752B08950F931F93CF93DF938D
:10577000EC019A01AB01662757FD6095762F0E94D8
:10578000752B8C01CE010E94EF2A800F911FDF91B3
:10579000CF911F910F9108952115310549F4DC0136
:1057A000ED91FC910190F081E02D642F0995089511
:1057B0000E94392B08959A01462F50E060E070E076
:1057C0000E94CC2B08959A01AB0160E070E00E942A
:1057D000CC2B08950F931F93CF93DF93EC010E947E
:1057E000CC2B8C01CE010E94EF2A800F911FDF91FC
:1057F000CF911F910F9108950F931F93CF93DF9334
:10580000EC019A01AB0160E070E00E94CC2B8C01AE
:10581000CE010E94EF2A800F911FDF91CF911F913F
:105820000F9108950F931F93CF93DF93EC019A018B
:10583000462F50E060E070E00E94CC2B8C01CE013E
:105840000E94EF2A800F911FDF91CF911F910F913E
:105850000895FC0124853585F901E05CFF4F8081C6
:105860009181F901EE5BFF4F20813181821B930B07
:105870008F7399270895FC0184859585FC01E05C70
:10588000FF4F40815181FC01EE5BFF4F2081318150
:105890004217530741F00190F081E02DE80FF91F06
:1058A000808190E008958FEF9FEF0895FC0184853B
:1058B0009585FC01E05CFF4F40815181FC01EE5B6E
:1058C000FF4F208131814217530779F0A081B181C8
:1058D000A80FB91F8C91208131812F5F3F4F2F730B
:1058E00033273183208390E008958FEF9FEF089551
:1058F000FC0181A1882329F0A489B5898C9186FFB8
:10590000FBCF11A20895CF93DF93FC012685378545
:10591000D901A05CBF4F8D919C91119701968F7317
:105920009927E901CE5BDF4F48815981841795079C
:10593000D9F30D90BC91A02DA20FB31F6C93A68537
:10594000B785A05CBF4F11969C938E93A689B789AB
:105950002C9181E090E0078C02C0880F991F0A9477
:10596000E2F7282B2C9381E081A30488F589E02DB0
:1059700080818064808381E090E0DF91CF91089501
:1059800008951F920F920FB60F9211242F933F93F9
:105990004F938F939F93EF93FF938091C00082FD6D
:1059A0001CC04091C600809188069091890601969E
:1059B0008F73992720918A0630918B06821793075F
:1059C00071F0E0918806F0918906E85BF94F408319
:1059D000909389068093880602C08091C600FF914B
:1059E000EF919F918F914F913F912F910F900FBE0B
:1059F0000F901F90189582EE95E00E94292C892B1C
:105A000011F00E94C02C08951F920F920FB60F92B2
:105A100011242F933F938F939F93EF93FF932091A4
:105A20004406309145068091460690914706281716
:105A3000390731F48091C1008F7D8093C10014C07B
:105A4000E0914606F0914706EC5FF94F2081809186
:105A500046069091470601968F73992790934706C3
:105A6000809346062093C600FF91EF919F918F91FE
:105A70003F912F910F900FBE0F901F901895A0E0AF
:105A8000B0E0E5E4FDE20C94C82EFC011382128222
:105A900088EE93E0A0E0B0E084839583A683B7838B
:105AA0008CEB93E091838083758764875787468763
:105AB000318B208B138B028BF58AE48AD78AC68AB6
:105AC000B18EA08E938E828E8F85848F8889858FEC
:105AD0008989868F8A89878F8B8980A3ECE00C94D3
:105AE000E42ECF92DF92EF92FF92CF93DF93EC01FF
:105AF0006A017B01411581EE580761057105F9F0D6
:105B0000EC89FD8981E090E008A002C0880F991F10
:105B10000A94E2F7808360E079E08DE390E0A701EA
:105B200096010E94812E2150310941095109569553
:105B3000479537952795211580E1380798F0EC892E
:105B4000FD89108260E874E88EE190E0A70196017B
:105B50000E94812E215031094109510956954795DE
:105B600037952795E889F9893083EA89FB8920836D
:105B700019A2EE89FF89408181E090E09C010C8CA4
:105B800002C0220F331F0A94E2F7422B4083EE89B2
:105B9000FF8940819C010D8C02C0220F331F0A94A3
:105BA000E2F7422B4083EE89FF8940819C010E8CF5
:105BB00002C0220F331F0A94E2F7422B4083EE8982
:105BC000FF8920810F8C02C0880F991F0A94E2F789
:105BD000809582238083DF91CF91FF90EF90DF90BB
:105BE000CF9008958F929F92AF92BF92CF92DF9203
:105BF000EF92FF920F931F9381E08F9385E08F9335
:105C000087E08F9383E08F9384E08F93E6EC8E2E72
:105C1000912CF2ECAF2EB12CA1ECCA2ED12CB0EC11
:105C2000EB2EF12C04EC10E025EC30E044E056E0E3
:105C300068E476E082EE95E00E943F2D0F900F9091
:105C40000F900F900F901F910F91FF90EF90DF90AA
:105C5000CF90BF90AF909F908F9008950E9472292F
:105C60000E94B022CBEFDCE20E9464252097E1F392
:105C70000E94FB2CF9CFA29FB001B39FC001A39F4C
:105C8000700D811D1124911DB29F700D811D112475
:105C9000911D08950E943B2EA59F900DB49F900DDD
:105CA000A49F800D911D11240895B7FF0C944A2ED6
:105CB0000E944A2E821B930B0895DB018F939F93C2
:105CC0000E944A2EBF91AF91A29F800D911DA39F6C
:105CD000900DB29F900D1124089597FB072E16F496
:105CE000009407D077FD09D00E94FF2E07FC05D055
:105CF0003EF4909581959F4F0895709561957F4FE3
:105D00000895A1E21A2EAA1BBB1BFD010DC0AA1FFC
:105D1000BB1FEE1FFF1FA217B307E407F50720F014
:105D2000A21BB30BE40BF50B661F771F881F991F8F
:105D30001A9469F760957095809590959B01AC01D8
:105D4000BD01CF010895052E97FB1EF400940E941B
:105D5000BA2E57FD07D00E94812E07FC03D04EF4C7
:105D60000C94BA2E50954095309521953F4F4F4F4A
:105D70005F4F089590958095709561957F4F8F4FF7
:105D80009F4F08952F923F924F925F926F927F9212
:105D90008F929F92AF92BF92CF92DF92EF92FF923B
:105DA0000F931F93CF93DF93CDB7DEB7CA1BDB0BE7
:105DB0000FB6F894DEBF0FBECDBF09942A8839888C
:105DC00048885F846E847D848C849B84AA84B98493
:105DD000C884DF80EE80FD800C811B81AA81B9819F
:105DE000CE0FD11D0FB6F894DEBF0FBECDBFED01B3
:105DF0000895EE0FFF1F0590F491E02D0994AA1B62
:105E0000BB1B51E107C0AA1FBB1FA617B70710F0A5
:105E1000A61BB70B881F991F5A95A9F780959095D7
:105E2000BC01CD0108958F929F92AF92BF92CF9205
:105E3000DF92EF92FF92CF93DF93EC01688179813B
:105E40008A819B81611571058105910521F464E2C8
:105E500079ED8BE597E02DE133EF41E050E00E94D2
:105E6000A32E49015A019B01AC01A7EAB1E40E94AB
:105E70004A2E6B017C01ACEEB4EFA50194010E94A7
:105E8000582EC60ED71EE81EF91EF7FE06C081E08A
:105E9000C81AD108E10880E8F80AC882D982EA82E3
:105EA000FB82C701B6019F77DF91CF91FF90EF9002
:105EB000DF90CF90BF90AF909F908F9008950E94F9
:105EC000132F089586E091E00E94132F08956093A8
:105ED00006017093070180930801909309010895CA
:105EE0002F923F925F926F927F928F929F92AF928A
:105EF000BF92CF92DF92EF92FF920F931F93CF93B7
:105F0000DF938B01EA016115710521F0DB018C93B0
:105F100011969C93209739F09E012250310923322B
:105F2000310508F0D8C07C016701BFEFCB1ADB0A4E
:105F30005601F7016080862D90E00E94A230892BE7
:105F400011F07601F1CFFDE26F120AC0570182E035
:105F5000A80EB11CD70111966C90772473940BC0D6
:105F6000BBE26B1207C05701E2E0AE0EB11CD701D5
:105F700011966C90712CCE018F7E892B89F4B0E341
:105F80006B1237C0F50180818F7D8835D1F4618037
:105F9000F2E0AF0EB11C872D8260782EC0E1D0E018
:105FA000CA30D10551F1C031D10521F0C830D10539
:105FB00099F409C0CC24CA94DC2CEC2CAFE0FA2E66
:105FC00022C0209769F7C8E0D0E0CC24CA94DC2C2A
:105FD000EC2CFFE1FF2E17C06FEF7FEFCB019E018E
:105FE000442737FD4095542F0E94812E69017A0184
:105FF0000AC02097A9F6CAE0D0E0E9E9CE2EDC2C51
:10600000EC2CE9E1FE2EF50160E020E030E0A90192
:106010004E01AA2497FCA094BA2C1F0170ED572EB4
:10602000560CA9E0A51570F48FEB860D8A3118F493
:1060300099EC592E06C08FE9860D8A3148F589EA18
:10604000582E560C852D90E08C179D070CF56F3F50
:10605000D9F0C216D306E406F50698F0C501B401DE
:106060000E945D2E9B01AC01852D90E0A0E0B0E088
:10607000280F391F4A1F5B1F281739074A075B077C
:1060800010F46FEF01C061E03196D1016C90C5CF83
:106090000115110551F0662311F0319703C071FE0F
:1060A00004C03297D801ED93FC9370FE07C0509561
:1060B0004095309521953F4F4F4F5F4F67FF10C080
:1060C00082E290E090938D0680938C066FEF7FEFD5
:1060D0008FEF9FEF07C060E070E080E090E002C0CB
:1060E000B901CA01DF91CF911F910F91FF90EF90FD
:1060F000DF90CF90BF90AF909F908F907F906F90E8
:106100005F903F902F900895FC0188279927E8948D
:1061100021912032E9F3293010F02E30C8F32B32D0
:1061200041F02D3239F4689404C00E94D630820FB9
:10613000911D219120532A30C0F31EF49095819532
:106140009F4F0895911150C0803219F089508550A9
:10615000D0F7089548EC53E00E94AF300895FA015B
:10616000A191B081009719F41097E1F0CD01DC0105
:10617000CD010D90002011F4C00113C0FB0121914D
:10618000222319F02015D9F7F3CFFB012191201517
:1061900019F41E92119606C02223C1F70D9000201B
:1061A000A1F7D001FA01A193B08308957AE0979FF7
:1061B000902D879F802D910D11240895F999FECF80
:1061C00092BD81BDF89A992780B50895262FF99937
:1061D000FECF1FBA92BD81BD20BD0FB6F894FA9ACA
:1061E000F99A0FBE01960895992788270895F89483
:0261F000FFCFDF
:1061F20000008E06200001000000FF0002000200E5
:10620200020002000200020002000200020002007C
:1062120002000200020002000200028025000005C6
:10622200400AA1204EA50020244EA52C2330C012E6
:1062320000001A400AA1204EA5001B1E27522C2343
:10624200308025000005400AA1204EA50020244EE2
:10625200A52C2330004B000006400AD0009D4900C7
:106262007B289D492C233000E1000005400A4501AE
:10627200D7DC03B81E0EBF00232E48E801008A4077
:106282000A6001555502AD1E20000023C801545872
:106292002074696D656F75742100596573004E6FC6
:1062A200002C00386368004E2F41002C205B005DFB
:1062B2002028002900486F70206368616E6E656C4B
:1062C200200020402000456E746572696E6720616F
:1062D20064617074697665206368616E6E656C20B6
:1062E20073656C656374696F6E2C207069636B698A
:1062F2006E673A007363616E6E6572206D6F6465DE
:10630200004E4F5420454E41424C45440053656E69
:1063120064696E672073657474696E677320746F45
:106322002052580A00526573657474696E6720734F
:10633200657474696E6773206F6E2052580A00414B
:10634200626F727465642065646974730A00696EB1
:1063520076616C69642073656C656374696F6E0045
:106362000D0A496E76616C696420696E70757420DD
:106372002D2064697363617264656421070053654B
:106382007474696E677320736176656420746F201C
:10639200454550524F4D0A005265766572746564E8
:1063A2002073657474696E67732066726F6D204521
:1063B2004550524F4D0A004C6F616465642066611E
:1063C20063746F72792064656661756C74730A0018
:1063D2004B657920616E64206368616E6E656C73D3
:1063E2002072616E646F6D697A65640A004F706530
:1063F2006E4C52536E6720545820737461727469E4
:106402006E672000206F6E20485720006D6F647504
:106412006C65206C6F636B65643F00342B3400380D
:1064220000382B340031320031322B340031360047
:1064320050504D0052535349005344410053434C72
:1064420000525844005458440041494E004C4245C1
:1064520045500053504B54524D0053425553005334
:10646200554D44004C4C494E440000070B0C101192
:106472001500B7012B032F033103350338033D0306
:10648200B7014003440349034D0351035503590324
:106492005D0363036A036F0374038D028D028D0231
:1064A2008D02160A1322312900000000832C882A4B
:0864B200292C562C3B2C782C00
:107E00000F92CDB7DEB7112484B714BE81FFF1D035
:107E100082E08093C00088E18093C10086E0809377
:107E2000C20080E18093C4008EE0CDD088249924E4
:107E3000CC24C394F5E0DF2EE1E1EE2E73E0F72EC3
:107E4000B6D0082F813479F4B2D08983C2D0898129
:107E5000823811F481E005C0813811F485E001C059
:107E600083E09ED09AC0823411F484E103C085344B
:107E700019F485E0B6D091C0853561F498D0082F0B
:107E800010E095D090E0982E8824802A912A880CC2
:107E9000991C82C0863521F484E0A3D080E0E1CF34
:107EA000843609F04CC083D082D0A82E80D0B82E62
:107EB00000E011E07CD0F80181938F01AE16D1F77C
:107EC00088D0FB2DF53489F4E0E0F1E00BC0F9999E
:107ED000FECF92BC81BC0894811C911C819180BD15
:107EE000FA9AF99AEA1598F358C08B2D863409F05E
:107EF00054C0F401F7BEE89507B600FCFDCFF401CD
:107F0000A0E0B1E02C9130E011968C91119790E0B7
:107F1000982F8827822B932B12960C01C7BEE895C9
:107F20001124329681E0A038B80761F7F401D7BE7A
:107F3000E89507B600FCFDCFE7BEE8952EC0843774
:107F4000F1F435D034D0182F32D0B82E42D0FB2DDA
:107F5000F63421F4F40105914F010CC0FB2DF534EA
:107F600049F4F999FECF92BC81BC0894811C911C04
:107F7000F89A00B5802F14D0115049F70EC08537FC
:107F800039F427D08EE10CD085E90AD08FE069CF93
:107F9000813511F488E017D01CD080E101D050CF9A
:107FA0009091C00095FFFCCF8093C600089580910A
:107FB000C00087FFFCCF8091C00084FD01C0A89560
:107FC0008091C6000895E0E6F0E098E19083808318
:107FD0000895EDDF803219F088E0F5DFFFCF84E10E
:107FE000DFCF1F93182FE3DF1150E9F7F2DF1F9166
:0E7FF0000895282E80E0E7DFEE27FF27099492
:027FFE0001057B
:0400000300007E007B
:00000001FF
